:100000000C94EB020C9408030C9408030C94EC1170
:100010000C944C360C9408030C941D360C94D72881
:100020000C9487310C9490280C9408030C940803CA
:100030000C940A360C947F280C9408030C94080343
:100040000C9408030C9408030C9408030C94080304
:100050000C9408030C9493360C9408030C94080336
:100060000C9408030C9408034D0D4F0D510D530DC6
:10007000550D570D590D5B0D5D0D840D870D8A0DC6
:100080008D0D900D930D960D990D9C0D291E2C1E16
:100090002F1E321E351E381E3B1E3E1E411E441EA4
:1000A0009A1F9D1FA01FA31FA61FA91FAC1FAF1F34
:1000B000C71FCA1FCD1FD31FD61FD01FD91FDC1FBC
:1000C000DF1FE21F20202320262029202C202F2084
:1000D000352032203820552058205B205E206120BA
:1000E000642067206D206A209C209F20A220A520EC
:1000F000A820AB20AE20B120B420B720BA20BD206C
:10010000C020C721C921CB21CD21CF21D121D3218D
:10011000D521D721D921C52120446F6E65210065E5
:1001200072726F723A00416420696E66696E69741A
:10013000756D00426C696E6B00556E6465726C691A
:100140006E650043572D5200435700312020204850
:100150007A0031302020487A0031303020487A004F
:1001600035303020487A00312020206B487A003129
:100170003020206B487A00313030206B487A0031D3
:100180002020204D487A00313020204D487A0053FD
:10019000706C697400537065656420005249542086
:1001A0000053656D690046756C6C005753505200E2
:1001B0004357004F4646004F4E200052696E67007D
:1001C0005469702000426F746800556C74696D61E9
:1001D0007469630049414D42494320420049414D01
:1001E0004249432041005374726169676874005347
:1001F000693533353141206572726F72005152504A
:10020000204C6162732C203230313900312E303174
:100210006100355720435720546376722000202F09
:100220003D3F2E2C7E7F06DB07557365206F72697C
:1002300067696E616C204943210052657365742EB5
:100240002E2E2000204D487A0053656C6563742083
:1002500062616E643A0053657474696E67207570EC
:100260002E2E2E00C00DED146C1B8827C436C846F8
:100270001C524E61746D0202020202020B06060657
:100280000B0B020302020003020300040107060134
:1002900001040100030002020201010201010B033B
:1002A0000307050302020203030303030301010121
:1002B0000002030203000302020001030104010122
:1002C000010403010002020002000002010B0B0105
:1002D000070101065369676E616C2067656E2E0029
:1002E0004672657175656E637900417564696F204A
:1002F00043682E3200417564696F2043682E3100D7
:10030000524620506F77657200566F6C7461676556
:100310000050726573732053656C656374210047E8
:10032000505320646174610043616C2073797320C1
:100330006F73630043616C20726566206F736300A6
:100340005068617365204869005068617365204C8E
:100350006F00492D512062616C005065616B204235
:1003600050460053797374656D2066727100526552
:100370006620667271005068617365204869206666
:100380007271005068617365204C6F206672710055
:10039000492D512062616C2066727100416C696761
:1003A0006E2066727100537572653F20656E7465CC
:1003B0007220313700466163746F727920727374F2
:1003C0002E00437573746F6D2073706C73680053E7
:1003D0002D6D6574657220737465700053686F7756
:1003E00020532D6D6574657200437572736F7220B2
:1003F0007374796C6500426174742E207374657037
:1004000000426174742E2066756C6C0042617474D5
:100410002E2073686F770044626C2E20636C6963D2
:100420006B005365742074696D65005753505220FA
:100430006C6F6361746F72005753505220706F7706
:10044000657200575350522063616C6C00537461A5
:100450007274004672616D65004672657175656EF5
:100460006379004D6F646500426561636F6E00459E
:100470006E61626C65206564697400456E61626CD2
:100480006520547800456E61626C652052780041A9
:100490006D706C2E206176672E0053706565642048
:1004A0006176672E004E6F69736520626C6E6B2EED
:1004B00000537472676874206D6F646500536964DB
:1004C00065746F6E6520766F6C0053696465746F38
:1004D0006E652066727100507261637469636500B5
:1004E00051534B004175746F205370616365004B2D
:1004F0006579657220576569676874004B65796531
:10050000722073776170004B657965722073706536
:100510006564004B65796572206D6F6465004357B3
:10052000206F6666736574004357206D6F646500C5
:100530005249542072617465005249540054756EDA
:100540006520726174650056464F20420056464F42
:1005500020410056464F206D6F64650052657065FE
:1005600061747300496E74657276616C004D6573D9
:100570007361676520005072657365742000536174
:1005800076652073657474696E67732100546573B2
:10059000742065717569706D656E7400416C696772
:1005A0006E6D656E74004F746865720042656163BC
:1005B0006F6E004465636F646572004B65796572A8
:1005C0000056464F004D6573736167657300507246
:1005D00065736574000011241FBECFEFD8E0DEBF45
:1005E000CDBF11E0A0E0B1E0E8EDFBE702C005906F
:1005F0000D92AC3EB107D9F724E0ACEEB1E001C0FA
:100600001D92A23FB207E1F70E94DA170C94EA3D6F
:100610000C94000000C000C000C000C000C000C0BA
:1006200000C000C0000008953C983D98449845984B
:1006300008953C9A08953C9AEDDF1DD008953D9AA7
:10064000E9DF3C98E7DF3D98E5DF3C9AE3DF13D034
:100650000895082E3C9ADEDF802D0DD0882311F0FE
:1006600002D0F8CF08953D9A3C9AD4DF3D98D2DF6E
:100670003C98D0DF08950894881F01C0880F59F076
:100680003D9A18F400003C9802C03C9A00C0C2DFBA
:100690003D98C0DFF3CF3D9A3C98BCDF3D98359B39
:1006A000FECF8827349981E0B5DF99270895882700
:1006B00001C081E071E03D9A3C98ACDF3D98AADF33
:1006C000359BFECF889434990894771FA0F73D9A04
:1006D000813011F03C9801C03C9A9CDF3D98359BDD
:1006E000FECF98DF872F992708959091B1039650F8
:1006F00081E0943008F080E00895CF93C1E0C0938A
:100700001A020E9475038823D9F08FEF0E94693680
:1007100080E00E94F12B81E00E94A6300E949E3072
:10072000809168008E7F8093680080917A00886055
:1007300080937A00C093700081E0CF910C941C32BA
:100740008091B1038C3061F480E00E947F3080E0C2
:100750000E94A63082E00E94DC0FCF910C94630FC0
:1007600080E00E947F3080E00E94A63081E00E94FD
:10077000DC0F1092800010926F00C09352048DEF36
:10078000809315021092160210921702109218020E
:100790001092190280917A00877F80937A0080916D
:1007A000B1038B3021F4C0938100CF91089587E08D
:1007B0008093810081E0CF910C94F12B10921A026A
:1007C00080E00E94F12B80E00E94A6300E94F50F8D
:1007D0008FEF0E946936EAE7F0E0808188608083CD
:1007E00081E08093700080E00C941C32CF92DF9205
:1007F000EF92FF92CF938FE40E940B1680915204E8
:10080000882331F0809115028D3F11F083E001C003
:1008100080E20E94181680915204882309F4D3C004
:1008200020915004309151048091EC019091ED01A0
:100830008217930750F46091500470915104681B23
:10084000790B6B01E12CF12C0DC0C0905004D090BD
:100850005104E12CF12C2FEFE21AF20AC81AD90A3E
:10086000E108F10880915004909151049093ED01BA
:100870008093EC0180E40E940B168091150221E028
:10088000280F8D3F08F097C03091B1033A3049F4FA
:10089000C11480E8D806E104F10418F48FEFE81AD7
:1008A000F80A8091160290911702A0911802B09157
:1008B0001902BC01CD016C0D7D1D8E1D9F1D609325
:1008C00016027093170280931802909319022093D6
:1008D00015023B3061F430E040E050E00E94643BA0
:1008E00069017A018FECE81A8EEFF80A1AC02430F9
:1008F00039F46B017C0128E6E21A2EEFF20A11C0EE
:1009000030E040E050E00E94643B69017A0186E6F5
:10091000E80EF11C82E0CC0CDD1CEE1CFF1C8A955D
:10092000D1F74BE0C701B6010E94AC3789E594E0EE
:100930000E94321680911502843009F044C088E18B
:1009400091E00E943E16809168008E7F809368003F
:1009500081E08093700080E00E94F12B80E00E9493
:10096000A6308091B1038B3059F4C0920404D09228
:100970000504E0920604F09207040E94DD1A0AC002
:10098000C092D003D092D103E092D203F092D3036D
:100990000E94E91A809123028823A9F00E94DE03B5
:1009A000109209041092230280E00E94C80A83E09A
:1009B0008093C70408C020931502CFE080E20E9414
:1009C0001816C150D9F78FEF80935204CF91FF9042
:1009D000EF90DF90CF9008950F931F938091430382
:1009E00090914403409116025091170260911802B1
:1009F00070911902480F591F611D711D4093160215
:100A00005093170260931802709319028091150297
:100A10008F5F893119F08093150248C0109215023A
:100A2000E091EE0181E08E0F8A019B010E2E04C041
:100A300036952795179507950A94D2F70133110536
:100A40002105310528F0E82FEDCFEE2361F1E150CB
:100A5000DB01CA010E2E04C0B695A7959795879520
:100A60000A94D2F780319105A105B10570F3E093A6
:100A7000EE018093160290931702A0931802B09390
:100A800019020E94AB178EE00E940B168091EE01B6
:100A90000E94271610921602109217021092180246
:100AA0001092190203C01092EE01E3CF1F910F9133
:100AB00008951092CA031092030481E080937D028E
:100AC0000E9482130C941516CF9310922802109254
:100AD00027021092200210921F028FEF90E0909355
:100AE0001E0280931D02809111048130A1F50E94A5
:100AF000E738C82F8091190490911A04A0911B0423
:100B0000B0911C046627782F892F9A2F27E731E0B0
:100B100040E050E00E94643B2093990330939A0395
:100B200040939B0350939C03CC2349F18CEA95E0BE
:100B30000E943E1680E20E9418168FE191E00E940A
:100B40003E1680E40E940B168C2F0E9417208DE227
:100B50008093550439C08091CA03882319F080918D
:100B6000FE030BC088EC90E09093B8038093B7032A
:100B70008CE590E00E94BF3D862F0E94F512809187
:100B8000CA03811107C08091EB0381110E941E29C5
:100B90000E94EC0C1092250210921B028FEF8093A2
:100BA0001C02109224028091230490912404A091AD
:100BB0002504B09126048093930390939403A0930B
:100BC0009503B0939603C0E08C2FCF91089591E0E8
:100BD0009093CA0390930304882319F09093A90378
:100BE00006C086E890E00E94B73D8093A90310926A
:100BF00011040E94640583E08093C7041092D5031A
:100C0000089580912402811110C080912304909155
:100C10002404A0912504B09126048093930390931B
:100C20009403A0939503B0939603809111048130AF
:100C300019F40E94F73A02C00E949F06882311F11E
:100C40008091CA03882389F08091A903882339F011
:100C500081508093A903811102C00C94590588E842
:100C600090E00E94BF3D6093D5030E94640580918F
:100C7000CA03811163C083E00E94DC0F81E080938E
:100C8000230208954091930350919403609195033A
:100C9000709196038091990390919A03A0919B0380
:100CA000B0919C03840F951FA61FB71F80939303D9
:100CB00090939403A0939503B093960380911104AD
:100CC000811107C08091A6039091970389130E9418
:100CD0005413209127023091280280911F02909195
:100CE0002002820F931F9093280280932702209165
:100CF0001D0230911E0282179307D0F0409193039A
:100D00005091940360919503709196034F5F5F4FEC
:100D10006F4F7F4F409393035093940360939503D9
:100D200070939603821B930B909328028093270263
:100D30008091CA03811102C00C94780C08958091AF
:100D4000250281110DC080911B02815080931B02EE
:100D5000811109C080912402811105C082E001C087
:100D600081508093250280911B028F3F09F065C05E
:100D700080912402882379F020912402215020932D
:100D800024023091EF013F3E09F03FC010921B0258
:100D90001092260248C090911C029F5F90931C0203
:100DA0002091B7033091B803A901490F511DCA0121
:100DB0000E94B73D8093EF01811102C081E0089548
:100DC00080910F040E94201F90911C028917B1F39B
:100DD0008091EF010E94951AE82FF0E0E05EFE4F4F
:100DE00020812093EF0187E030E09FEF980FA90169
:100DF000082E02C0559547950A94E2F740FF02C0BD
:100E0000892FF3CF80932402B7CF81E090E001C017
:100E1000880F2A95EAF7832349F083E080931B0229
:100E200081E0809326021092220207C081E0809325
:100E30001B02809322021092260280911B028111D4
:100E400004C0109222021092260280912202811187
:100E500007C081E090912602911103C080E001C09B
:100E600081E00E94961280E00895CF938091020461
:100E7000823079F08091B1038D3F59F08C3F59F069
:100E80008091BF039091C0038115904831F0C7E075
:100E900005C0CBE003C0C9E001C0C0E080E48C0F16
:100EA0000E940B16EC2FF0E0E15DFD4F80810E9467
:100EB000181681E08C0FCF91089580916202A0E214
:100EC000B1E0E0E09D91981719F0EF5FEA32D1F7B9
:100ED0008EEF80936202EA3010F480E303C0E432C4
:100EE00018F487E38E0F0895EA3229F0F0E0E65017
:100EF000FE4F849108958AE20895EFE2F2E080E2E5
:100F0000819392E0EF33F907D9F7089580912E028B
:100F100090915602981779F08F5F803119F0809385
:100F20002E0202C010922E02E0912E02F0E0ED5946
:100F3000FD4F8081089580E0089590912E02809168
:100F40005602981799F090912E02809156029817A8
:100F500079F0EFE2F2E08181819382E0EF33F807EC
:100F6000D1F70E94860780933E02EDCF80E008957E
:100F700081E00895CF93DF93C82FD62F8091090485
:100F80008823D1F08091AA03882351F18091AB038B
:100F9000813051F4E0917E02F0917F02E75AFB4FDD
:100FA000C0830E940F281CC08230D1F48C2F0E9475
:100FB00067388111EFCF14C080916002882381F0DF
:100FC000809156028F5F803119F08093560202C0E3
:100FD00010925602E0915602F0E0ED59FD4FC083A9
:100FE000DD2381F080916102882321F081E09091DE
:100FF000B20303C081E09091BE03911101C080E073
:1010000080936002DF91CF910895CF92DF92EF92AB
:10101000FF9281E0809361022091FE0330E040E086
:1010200050E060EB74E080E090E00E94643B20932D
:10103000490230934A0240934B0250934C02A3E082
:10104000B0E00E94A23B60934E0270934F028093E7
:10105000500290935102DC01CB01820F931FA41F19
:10106000B51FB695A7959795879580934502909360
:101070004602A0934702B093480281E09091B203E8
:10108000911101C080E0809360028EEF8093620234
:101090001092400210924D02FF90EF90DF90CF909F
:1010A00008951092610208954F925F926F927F921D
:1010B0008F929F92AF92BF92CF92DF92EF92FF9268
:1010C0008091770290917802A0917902B0917A0292
:1010D0000496A11DB11D8093770290937802A0938E
:1010E0007902B0937A02E0904303F0904403809138
:1010F000B10387FD06C080916102811102C00E9488
:1011000005089091A60380916102992329F081112D
:1011100041C00E9405083EC09091F401992389F0D6
:101120008091770290917802A0917902B0917A0231
:101130008093F0019093F101A093F201B093F30139
:1011400029C0882339F18090770290907802A0908E
:101150007902B0907A028091F0019091F101A09112
:10116000F201B091F301881A990AAA0ABB0A2091E8
:10117000490230914A0240914B0250914C02AEE03C
:10118000B0E00E94A23B681579058A059B0510F422
:10119000109261028091A6038093F4014091610254
:1011A00041113AC0E0910001F0910101EE15FF05F7
:1011B000F0F4209102013091030160910A042E1590
:1011C0003F0548F4C701821B930B70E00E94503B1F
:1011D000260F371F08C0C9018E199F0970E00E94B1
:1011E000503B261B370B3093030120930201809163
:1011F0000201909103018E179F0720F4F0930301E1
:10120000E0930201809102019091030196958795E8
:101210008E159F0520F481E080935B0202C010923E
:101220005B0280915B0290914D02891799F0C0900A
:101230007702D0907802E0907902F0907A02C09222
:101240005202D0925302E0925402F09255024111A0
:1012500024C025C0411121C0C0907702D0907802EF
:10126000E0907902F0907A0240915202509153023C
:101270006091540270915502C41AD50AE60AF70A21
:101280004091CF0350E060E070E04C155D056E05C5
:101290007F0528F490912D02891380932D022091CF
:1012A0002D0280914002281709F4FBC0C0907702FC
:1012B000D0907802E0907902F0907A028091520208
:1012C00090915302A0915402B0915502222311F142
:1012D0008093410290934202A0934302B093440250
:1012E0008091570290915802A0915902B0915A02F0
:1012F000C81AD90AEA0AFB0AC0925C02D0925D02BF
:10130000E0925E02F0925F028091F501882309F479
:1013100091C0C5C08093570290935802A093590280
:10132000B0935A028091410290914202A0914302EF
:10133000B0914402C81AD90AEA0AFB0AC0922902EB
:10134000D0922A02E0922B02F0922C02D701C60121
:101350004E97A109B109873D9140A105B10508F05B
:10136000F1C04090BB03842C912C81E0881A910835
:10137000092C000CAA08BB08512C612C712C60911F
:101380004502709146028091470290914802A50162
:1013900094010E94343B6C0D7D1D8E1D9F1DA30189
:1013A00092010E94643B2093450230934602409391
:1013B000470250934802C216D306E406F506E8F445
:1013C0006091490270914A0280914B0290914C02C7
:1013D000A50194010E94343B6C0D7D1D8E1D9F1D47
:1013E000A30192010E94643B2093490230934A0278
:1013F00040934B0250934C02A5C060914E027091F5
:101400004F028091500290915102A50194010E94D7
:10141000343B6C0D7D1D8E1D9F1DA30192010E940A
:10142000643B20934E0230934F02409350025093FE
:10143000510288C08090490290904A02A0904B02CD
:10144000B0904C02A5E0B0E0A50194010E94A23B3F
:101450006C157D058E059F0540F40E945D0760E0D8
:101460000E94BA0761E080E218C080914E0290911C
:101470004F02A0915002B0915102880D991DAA1DF2
:10148000BB1DB695A795979587958C159D05AE05BF
:10149000BF0528F40E945D0761E00E94BA07109220
:1014A000F50180912D02811138C040917702509151
:1014B00078026091790270917A028091570290913E
:1014C0005802A0915902B0915A02481B590B6A0B5D
:1014D0007B0B80914E0290914F02A0915002B091EF
:1014E000510222E0880F991FAA1FBB1F2A95D1F72E
:1014F00084179507A607B70780F48091F50181113D
:101500000CC00E945D0760E00E94BA0761E080E2C3
:101510000E94BA0781E08093F50180915B0280937D
:101520004D0280912D0280934002FF90EF90DF905A
:10153000CF90BF90AF909F908F907F906F905F9073
:101540004F9008954091490250914A0260914B0298
:1015500070914C0280914E0290914F02A0915002E6
:10156000B0915102480F591F6A1F7B1F76956795EE
:101570005795479580916202C416D506E606F70690
:1015800010F4880F02C0880F8F5F8093620287CFAC
:10159000CF93C82F8091C20390917B02891B9091B9
:1015A0007E02890F0E940B16CC2341F08091CB0361
:1015B000813011F48DE003C08EE001C08CE0CF914A
:1015C0000C94F5158091B1038D3F21F48091FC03BB
:1015D0008F5B08C09091080181E0923008F480E0B0
:1015E0009F5F890F0E940B168EE00C94F515809179
:1015F000BF039091C00397FD12C08DE20E941816A0
:101600002091BF033091C00380E090E8A0E0B0E0FB
:10161000BC01CD01621B730B810991090FC08BE2E4
:101620000E9418166091BF037091C003CB01A0E027
:10163000B0E0BC01CD0170588109910946E00E94DB
:10164000AC3789E594E00C94321680E40E940B16C6
:101650008CE991E00E943E160E94F70A0E9408164B
:101660000E944D160C94E20A80E40E940B1685E954
:1016700091E00E943E1660E08091FE030E949D165C
:101680000E9408160C944D164BE00E94AC378091D6
:101690005904803319F480E2809359041092620453
:1016A00089E594E00C943216CF92DF92EF92FF928C
:1016B000CF93DF93C82FD62F69017A010E940B16B2
:1016C000D11102C084E001C085E00E941816C70154
:1016D000B6010E94440B8091CE03882391F0C11182
:1016E00010C08091CD03811103C080E20E941816C2
:1016F00080E5DF91CF91FF90EF90DF90CF900C9439
:101700001816DF91CF91FF90EF90DF90CF90089562
:10171000A0918002B0918102B7FF11C0BF7028EA8A
:1017200035E24AE050E00E94A23B20E034E840E08D
:1017300050E00E94643B30938102209380028091AC
:101740000901883009F04AC08091B10381111AC0A3
:1017500080E40E940B1660918002709181026B5FA1
:101760007F4F80E090E047E00E94AC378EE28093AC
:101770005B0480E280935E0486E580935F041092B0
:10178000600428C0813051F580E40E940B16A091BE
:101790008002B0918102A657BD4F9D010E948C3BF3
:1017A00028E334E441E050E00E94643BCA01B901FF
:1017B0006B5F7F4F8F4F9F4F46E00E94AC378EE2AA
:1017C00080935A0480E280935D0487E580935E04F1
:1017D00010925F0489E594E00C94321640910D0458
:1017E00050910E0426E0249FC001259F900D1124E6
:1017F0002091F0033091F1038217930718F4281B0E
:10180000390B02C020E030E06091800270918102CB
:1018100080E02617370730F4873021F0240F351F7A
:101820008F5FF7CF9091F601981721F08093F60122
:101830000C94CB160895809102048230C9F4209153
:10184000D8033091D9034091DA035091DB0360E073
:1018500080E00E94540B2091B3033091B403409177
:10186000B5035091B60361E080E40E94540B2AC096
:1018700081110AC02091D8033091D9034091DA0335
:101880005091DB0360E00AC02091B3033091B403B0
:101890004091B5035091B60361E080E00E94540B83
:1018A00080E20E9418168091BF039091C0038115B9
:1018B000904841F080E40E940B160E94F70A80E2F3
:1018C0000E9418168091FD03882339F00E94880B2E
:1018D0008FE00E940B1686E004C08FE00E940B167A
:1018E00080E20E9418160E94E20A10927D0208957A
:1018F00080E40E940B168CE00E94F5158091110483
:10190000813031F580912402813011F547E050E0BB
:1019100068EE73E089E594E00E94A73D89E594E0D4
:101920000E94321680E20E94181645E050E06FEEE9
:1019300073E089E594E00E94A73D89E594E00E9468
:10194000321680E20E9418168091C7030C94271665
:10195000089580915904882319F0813021F0089569
:1019600088E491E002C083E491E00C943E168091FB
:101970005904882319F0813021F0089589E391E01A
:1019800002C083E391E00C943E16809159048823B1
:1019900019F0813021F0089586EA91E002C081EAD1
:1019A00091E00C943E1680915904882319F087EB3E
:1019B00091E002C083EB91E00C943E1680915904B3
:1019C000882319F0813021F0089580EB91E002C066
:1019D0008BEA91E00C943E1680E00E940B16609119
:1019E000F8037091F9038091FA039091FB034BE0A7
:1019F0000E94AC3789E594E00E94321680E20E9492
:101A0000181680911104809359040E94DE0C809175
:101A10001104811107C080E20E9418168091FE0314
:101A20000C94271680E20C9418168091590481308A
:101A300049F028F0823049F0833051F0089586EE65
:101A400091E008C08DED91E005C084ED91E002C009
:101A50008AEC91E00C943E1680915904813039F063
:101A600018F0823039F0089585EC91E005C080ECE3
:101A700091E002C08BEB91E00C943E1680E40E9452
:101A80000B16E09159048E2F90E089309105C0F437
:101A9000FC01EC5CFF4F0C94863B80E50FC08CE3AF
:101AA0000DC088E20BC08EE109C084E107C081E16E
:101AB00005C08FE003C08CE001C08AE00E942716B9
:101AC0008DE60C94181680915904813051F038F04D
:101AD000823051F48FE891E00E943E1605C081E407
:101AE00001C082E40E9418160E9408160C944D163C
:101AF000E09159048E2F90E08930910508F5FC01A2
:101B0000E35CFF4F0C94863B87E891E017C08FE7BA
:101B100091E014C087E791E011C08FE691E00EC01C
:101B200087E691E00BC080E691E008C089E591E08E
:101B300005C082E591E002C08BE491E00C943E1672
:101B4000089580915904811105C086E291E00E94B8
:101B50003E1603C060E00E949D160E9408160C9479
:101B60004D160E94261F80915904882341F010923F
:101B7000690489E594E00E94321680E0089581E0CE
:101B800008950F931F93CF93DF9380E40E940B1669
:101B90008091AB0381114DC080910901823061F4C5
:101BA0008091B103811103C00E94630D3AC0863059
:101BB000B1F40E94A90C35C08330C9F48091B103FF
:101BC000853019F40E94C50C2CC0811103C00E94FD
:101BD000150D27C0893029F50E942C0D22C08330B5
:101BE00019F40E94780D1DC08530D9F4FACF8130E8
:101BF00039F48091B1038D30A1F40E94A10D11C080
:101C0000853039F48091B103813059F40E94DE0CA3
:101C100008C0863031F48091B103843011F40E9401
:101C2000B70C0E940816DF91CF911F910F910C9471
:101C30004D16833031F4DF91CF911F910F910C94A9
:101C4000D30CC0917B02D0917C02C75ADB4F00E1DC
:101C500010E08991882329F00E941816015011097B
:101C6000C1F7DF91CF911F910F91089581E080938B
:101C70007D0208952F923F924F925F926F927F92D2
:101C80008F929F92AF92BF92CF92DF92EF92FF928C
:101C90000F931F93CF93DF9300D000D0CDB7DEB763
:101CA000409004015090050160900601709007017A
:101CB000C82ED12CCC0CDD1CE12CF12C212C312C8C
:101CC00019821A8200E010E01C821B8298014C816C
:101CD0005B81C301B2010E94DF3C910149815A81BD
:101CE0000E94B53B4B015C01F601EE0DFF1DEE5766
:101CF000FD4F60817181072E000C880B990B0E94AB
:101D0000533CA50194010E94B63B4B015C0182E06B
:101D1000E80EF11C18018C8189838B818A8380E60F
:101D2000E816F10421F08401AC82BB82CFCF980188
:101D30004C815B81B401C5010E94DF3CA30192018B
:101D40000E94DF3C6B017C019401A501B401C50137
:101D50000E94DF3C4B015C0198014C815B81B80122
:101D60008C819B810E94DF3C9B01AC01C501B401C9
:101D70000E94B63BA70196010E94B53B0E94523DCE
:101D80000E94223C70934403609343030F900F9092
:101D90000F900F90DF91CF911F910F91FF90EF90D7
:101DA000DF90CF90BF90AF909F908F907F906F907B
:101DB0005F904F903F902F900895909159039F5FAF
:101DC000903119F09093590302C010925903E09199
:101DD0005903F0E0E75BFC4F80830895FA01D901D5
:101DE000118210821C92813049F56330B9F040F4C1
:101DF000613071F0623009F044C028E733E01AC066
:101E0000653091F070F06630E1F525E433E012C002
:101E10002FE633E03183208396E032C02EE533E0B5
:101E200005C026E733E006C02CE733E0318320838A
:101E30009FE026C0318320838C9323C0823029F415
:101E40006230F9F421E933E00DC0883029F46730BD
:101E5000C1F42EE833E011C0843099F4623031F4DB
:101E60002AE733E03183208391E00AC0643048F0F0
:101E70006370633031F42AE533E03183208392E0EC
:101E80009C9320813181232B29F090916E03892B23
:101E900080936E0308950F931F93F9019081DB01E6
:101EA000A90FB11D2C91281309C09F5F9083933017
:101EB00031F4D8014C93108281E002C0108280E09E
:101EC0001F910F91089580E40E940B1680916E037C
:101ED00080FF05C088E793E00E94321603C08DE2C0
:101EE0000E94181680E20E94181680916E0381FFEE
:101EF0000FC080919103823319F48AE491E00AC003
:101F0000833319F48DE491E005C080E591E002C0CF
:101F100083E591E00E94321680E20E94181686E660
:101F20000E94181680916E0383FF10C080918F036A
:101F3000811103C080E30E94181680918E030E94D5
:101F4000181680918F03882339F004C08DE20E9417
:101F500018168DE20E94181680E20E94181684E777
:101F60000E94181680915D0390916E039823A9F04A
:101F70000E94271680E20E94181683E70E94181616
:101F800060915D0370E080914703909148030E9447
:101F9000503B862F0E94271604C086E591E00E94E0
:101FA00032160E940816803520F480E20E9418162E
:101FB000F8CF10926E03089580938C030E9404362C
:101FC0008091680081608093680010926B0080911E
:101FD0008C03813031F480916B00806180936B00C1
:101FE00008958DED9EE00C94E0310E94D8310E945E
:101FF000DD3510928C03E8E6F0E080818E7F8083EF
:1020000010926B000895CF93DF9300D000D01F9201
:10201000CDB7DEB780917803813409F0ABC0409131
:102020007D0350E04053510920917C0330E0205360
:1020300031096AE0629FC001639F900D1124840FF3
:10204000951F97FD01969595879560914503653499
:1020500011F4865B03C099E4981B892F89838091D2
:102060005E03E0917603EE3411F4865E03C099E7D7
:10207000981B892F8A8380917E0390E0C0977AE035
:10208000749F9001759F300D1124820F931F97FD4F
:10209000019695958795653431F46AE00E94443B3A
:1020A000905D9B8306C06AE00E94443B89E3891BE4
:1020B0008B8390915F03EE3411F49C8303C089E617
:1020C000891B8C831D82CE0101960E94D23881111A
:1020D00026C045E050E06FEE73E089E594E00E9491
:1020E000A73D99818091590498130FC09A818091DE
:1020F0005A0498130AC09B8180915B04981305C011
:102100009C8180915C04981751F045E050E06FEE9F
:1021100073E0CE0101960E94C53D0E94E7384091D0
:102120007303440F4056842F880F880F480F809107
:1021300074038053480F60917103660F6056862FB9
:10214000880F880F680F809172038053680F809109
:102150006F03880F8056982F990F990F890F9091D0
:1021600070039053890F0E94B3298091210281113D
:102170000E941E2980918C03823019F40E94630F03
:1021800009C0833039F40E94F50F8AE08093B103CF
:102190000E947D030F900F900F900F900F90DF9192
:1021A000CF9108950F931F93CF93C82F8091000272
:1021B00081113DC08091FF018C278093FF0100E0D9
:1021C00012E02EEF31E041E06BE571E08C2F0E94D0
:1021D0004B0F882359F01092FE011092FD011092CE
:1021E000FC011092FB011092FA01DAC000E012E04B
:1021F0002DEF31E042E06FE571E08C2F0E944B0F34
:102200008111E9CF2CEF31E048E063E671E08C2FDB
:102210000E944B0F8111DFCF2BEF31E044E067E6E6
:1022200071E08C2F0E944B0F8111D5CFB9C0C43201
:1022300049F4109200021092FE011092FA011092DD
:10224000FF01AEC02091FA01CC3219F0CA3209F078
:1022500059C08091F8019091F901009769F040917F
:10226000FE013091F701FC01431718F4E40FF11D52
:1022700002C0E30FF11D108280910002843061F5ED
:10228000243050F1822F8370833031F5273051F4A0
:1022900080917A03813331F41092480310924703FE
:1022A00010925D03E091F801F091F901808188239B
:1022B00099F08AE593E00E947638209147033091A7
:1022C0004803620F731F7093480360934703809124
:1022D0005D038F5F80935D036091FA016F5F609390
:1022E000FA011092FE0127EF31E048EF51E08091B2
:1022F00000020E94EE0ECA3211F48EEF11C08091DE
:10230000FF014BC02E3F79F48C2F0E946E389091C4
:10231000FF0120E1829F901911249093FF018FEF1C
:102320008093FA013DC02F3FE1F48C2F0E946E385C
:102330009091FF01981B9093FF011092FA018091F8
:102340000002992339F0809590916E038923809340
:102350006E0326C0813021F5CF911F910F910C940F
:1023600003102091F8013091F9018091FF012115AE
:10237000310599F09091FE014091F701941768F4AE
:102380008C278093FF01F901E90FF11DC083809133
:10239000FE018F5F8093FE0103C0C827C093FF0139
:1023A000CF911F910F91089580918D0390915903C2
:1023B000891789F08F5F803119F080938D0302C0F7
:1023C00010928D03E0918D03F0E0E75BFC4F80817C
:1023D0000E94D210E9CF08951F920F920FB60F926C
:1023E00011242F933F934F935F936F937F938F931A
:1023F0009F93AF93BF93EF93FF9380918C038130B2
:1024000069F48091840090918500909351048093A9
:10241000500483B180718093520402C00E947231D3
:10242000FF91EF91BF91AF919F918F917F916F91AC
:102430005F914F913F912F910F900FBE0F901F9082
:102440001895CF93C82F0E94711A882371F180913B
:10245000A303882351F1C11115C040912304509169
:1024600024046091250470912604809103029091C8
:102470000402A0910502B091060284179507A607F1
:10248000B70798F480E00E94FC3180E00E94283277
:1024900080E00E947F3081E00E9422321092A303EC
:1024A00080916F008B7F80936F00CF910895CF92C2
:1024B000DF92EF92FF922091CC036091190470910A
:1024C0001A0480911B0490911C04C0902304D090A6
:1024D0002404E0902504F0902604222381F020912A
:1024E000FE0330E040E050E00E94643BA0E6B0E034
:1024F0000E94A23B2AE030E040E050E004C024E625
:1025000030E040E050E00E94643BC20ED31EE41E67
:10251000F51EC0920302D0920402E0920502F092EE
:102520000602FF90EF90DF90CF900895CF93C82FD1
:102530000E94FC310E94711A811114C0809109011E
:10254000883081F0C093A303CC2311F080E001C058
:1025500081E00E94223280E00E94283280E00E94C6
:102560007F3039C0CC2379F180E00E942232809103
:10257000A30381110AC08091CE03811103C081E0C1
:102580000E947F3081E08093A3038091CE0381116C
:1025900003C081E00E9428328091B903811104C0F8
:1025A00080910304882361F08FEF9FEFDC0180931B
:1025B000030290930402A0930502B09306020BC09D
:1025C0000E94571208C08091020281110E94571286
:1025D00080E00E9428328091A60380939703C093E5
:1025E000A603C0930202CF910895CF92DF92EF929B
:1025F000FF920F931F93282F30E040E050E060914E
:10260000190470911A0480911B0490911C040E947B
:10261000643BACE0B0E00E94A23B2AE030E040E046
:1026200050E00E94643BCA01B901209399033093A2
:102630009A0340939B0350939C0320910004309194
:1026400001046901E12CF12C243F314068F410921F
:102650009E0304EF11E020E030E0A90198012C195D
:102660003D094E095F0909C021E020939E03A7019F
:102670009601245F3140410951090E94343B28EE04
:1026800033E040E050E00E94643B20939F0330938E
:10269000A0034093A1035093A2031F910F91FF90B9
:1026A000EF90DF90CF9008950F931F9390919E032A
:1026B0004091930350919403609195037091960318
:1026C00000919F031091A0032091A1033091A203D8
:1026D000882339F0992339F0400F511F621F731F6F
:1026E00006C09923C9F3401B510B620B730B409337
:1026F00093035093940360939503709396031F91F3
:102700000F9108958091FE030E94F5128091230499
:1027100090912404A0912504B09126048093930302
:1027200090939403A0939503B09396038091F30341
:10273000811103C082E08093980308954F925F92C5
:102740006F927F928F929F92AF92BF92CF92DF92C1
:10275000EF92FF920F931F93CF935091F3038091C9
:10276000990390919A03A0919B03B0919C030091CF
:102770009303109194032091950330919603552370
:10278000F9F0409198034423D9F0109298034091B6
:10279000A5034770A9F4AC01BD01440F551F661F86
:1027A000771FD901C801840F951FA61FB71F8093FB
:1027B000930390939403A0939503B0939603C1C0A1
:1027C000C0902304D0902404E0902504F0902604C7
:1027D00026013701401A510A620A730A4C015D0151
:1027E000880C991CAA1CBB1C84149504A604B7046D
:1027F00028F48C0D9D1DAE1DBF1D04C0800F911FC0
:10280000A21FB31F8093930390939403A093950307
:10281000B093960351110EC080919803813051F40A
:102820008091A503877019F01092980303C082E08D
:1028300080939803809101028823F1F08150809366
:10284000010281117EC00E9496128091A5038C7FA7
:102850008093A503809101020E94541381E080932C
:1028600098038091B903813009F06BC08091A50372
:10287000877E8093A50365C09091B9038091A503DD
:10288000913041F4282F28742834D1F0282F207358
:10289000203359F082FF18C020919D03213051F45C
:1028A000933019F092E090939D0393E0909301028E
:1028B0008B7D2DC0933019F091E090939D0391E0B2
:1028C000909301028B7B17C080FD0FC081FF07C072
:1028D00093E09093010292E090939D0317C0923091
:1028E000C1F4282F2874283441F491E090939D037B
:1028F000909301028F7B80620DC0282F20732033BC
:1029000041F490939D0393E0909301028F7D806446
:1029100001C08F798093A5038091A503877E809362
:10292000A503809101020E949612C0910102CC235E
:1029300019F08C2F0E94541381E0C11180E0809324
:10294000A403CF911F910F91FF90EF90DF90CF9054
:10295000BF90AF909F908F907F906F905F904F90BF
:102960000895CF92DF92EF92FF92CF938091CA03A6
:102970008111BDC0809103048111B9C080911A02F8
:102980008111B5C00E94711A811104C08091B103F8
:1029900087FDADC00E949933C82F0E94B1332091AA
:1029A000B903211110C0C11106C091E0811101C00D
:1029B00090E0892F01C081E0CF91FF90EF90DF90F0
:1029C000CF900C949612C0902304D0902404E090F1
:1029D0002504F09026044091930350919403609154
:1029E0009503709196034C155D056E057F0510F0FB
:1029F00030E008C090919803992319F091E09093EA
:102A0000A40331E0C1110CC081111EC0223051F16C
:102A10008091A503887F8093A50310929D033FC0FA
:102A20009091A503882319F09C7F946024C091FFA6
:102A300019C09C7F94609093A503233009F451C082
:102A400092E090939D034DC09091A50390FF0AC022
:102A50009C7F94609093A5032330E1F081E0809304
:102A60009D0318C09091A403992381F0CC2331F0E9
:102A70009091A50391609093A50333C0882379F0CA
:102A80008091A50382608093A50304C0C11129C071
:102A9000882329F08091A50380618093A5033111DB
:102AA0000E949E138091F303811121C080919803AD
:102AB0008230E9F48091A5038770C9F010929803E1
:102AC0008091230490912404A0912504B0912604C0
:102AD0008093930390939403A0939503B0939603EC
:102AE00006C09091A50398609093A503D1CFCF9194
:102AF000FF90EF90DF90CF9008955C9A00C05C98B3
:102B000008950F931F9381E00091230410912404F2
:102B1000209125043091260440910702509108022B
:102B20006091090270910A0240175107620773070A
:102B300008F080E01F910F910895CF93C82F0E9455
:102B4000BB298091230490912404A0912504B09185
:102B500026048C0F911DA11DB11D80930702909337
:102B60000802A0930902B0930A02CF9108951F931F
:102B7000CF93DF93D82F162F409123045091240434
:102B800060912504709126048091070290910802BB
:102B9000A0910902B0910A0284179507A607B7070A
:102BA00018F00E94BB29E8CFCBB1C07F8C2FD7FD96
:102BB0008860D6FD8460D5FD8260D4FD8160D3FD40
:102BC000C860D2FDC460D1FDC260D0FDC1608BB9C8
:102BD000112311F0449A01C044980E947D15CBB98D
:102BE000DF91CF911F910C947D15CF93C82F60E09A
:102BF0000E94B715C43010F487E201C082E0CF9183
:102C00000C949D1561E00E94B71582E00C949D150F
:102C10008091A7030895CF93C82F80E88C0F0E945E
:102C2000F515C093A703CF91089581E00C94F51595
:102C300061E00E94B71582E00E949D158091A70374
:102C40008F5F8093A7030895805D0C941816CF932F
:102C50006AE00E94443BC92F0E9424168C2FCF911A
:102C60000C942416CF93DF93EC018991882319F0FB
:102C70000E941816FACFDF91CF910895CF93DF937A
:102C8000FC018491EF012196882321F00E941816FF
:102C9000FE01F7CFDF91CF910895CF93C82F809198
:102CA000A703C81719F08C2F0E940B16C03140F4EF
:102CB0008091A703803160F480E20E941816F8CF5B
:102CC0008091A703803520F480E20E941816F8CF87
:102CD000CF91089580E70E94F51580E00E940216CA
:102CE00082E00E94021686E00E9402168EE00E9498
:102CF00002168EE10E9402168EE00E94021686E005
:102D00000E94021682E00E94021680E00E940216D3
:102D100081E00E94021681E00E94021685E00E9476
:102D2000021689E00E9402168FE10E94021688E0D6
:102D30000E94021684E00C9402160F931F93CF9307
:102D4000DF93D62F082F10E0843640F0CCE9C80F6F
:102D5000C43638F0C8E3C80F82E004C0C82F80E052
:102D600001C081E00436110510F00E94241680E0B5
:102D700090E0CA3018F0CA500196FBCF0A30110516
:102D800008F4D1110E9424168C2FDF91CF911F914E
:102D90000F910C942416CF93DF93D82F80E70E94D5
:102DA000F5158EE00E940216C6E0DC1710F08FE1E8
:102DB00001C081E10E940216C150B9F78FE1DF9195
:102DC000CF910C940216CF93DF933C9A549A509A69
:102DD000519A529A539A80E49CE90197F1F7599AD3
:102DE000589A0E947D1580E891E60197F1F70E94BC
:102DF0007D15C0E4D1E0CE010197F1F70E947D1569
:102E0000CE010197F1F758980E947D152197F1F7AF
:102E100088E20E94F51588E00E94F5150E941516BB
:102E200086E00E94F5158CE00E94F51580E0DF91A8
:102E3000CF910C94CB16CF9380E40E94F515C8E097
:102E400080E10E940216C150D9F7C23010F084E12F
:102E500001C080E10E940216CF5FC830B1F7C0E028
:102E6000C23010F085E101C080E10E940216CF5F00
:102E7000C830B1F780E00E9402168AE00E94021674
:102E80008FE10E9402168FE10E9402168FE10E94DC
:102E900002168EE00E94021684E00E94021680E074
:102EA0000E9402168CE00E94021682E10E94021625
:102EB0008EE10E94021682E10E94021682E10E94C7
:102EC000021680E00E94021680E00E94021680E056
:102ED0000E9402168CE10E94021682E10E940216F4
:102EE0008CE10E94021682E10E9402168CE10E948F
:102EF000021680E00E94021680E00E94021680E026
:102F0000CF910C940216611103C08BE00C940B1648
:102F100070E061507109962F990F690F262F30E0EC
:102F2000F9013296482F50E0E417F50714F482E0D7
:102F30000FC0681710F080E20BC02F5F3F4F4217A1
:102F4000530711F480E004C0E417F50719F481E099
:102F50000C9418160895FF920F931F93CF93DF934D
:102F6000F82E80E40E940B16C2E0D0E00F2D10E096
:102F7000C017D10714F482E011C08C2F82508F1536
:102F800010F080E20BC0CE0101970817190711F469
:102F900080E004C00C171D0719F481E00E94181688
:102FA0002396C233D10521F7DF91CF911F910F9165
:102FB000FF90089585E085BD0E94E4350E94E316E8
:102FC0000E9415160E94BA1A0E947D0781E00E9495
:102FD0002232789480E480937C008FEE80937A0094
:102FE00085EF93E00E94B73DC82F811109C082E1AF
:102FF00092E00E943E168CE092E00E943E1605C0D0
:103000008AE00E94B10D8111F2CF80E40E940B167C
:10301000C11105C08DEF91E00E943E1605C08BE006
:103020000E94B10D8111F6CF84E180935604809106
:103030005604882359F080E00E94BB3880916000DC
:103040008111FCCF809156048150EFCF0E94CB1CA0
:103050000E9415160E941B1786EC90E00E94B73D57
:10306000893018F00E94CD1B03C082E08093C70412
:10307000D0E0712C00E0812C10E0C12CD12C760125
:10308000312CA12C912C5AE0552E44244A9460E313
:10309000662E8091B1038B3F51F480912704652DFA
:1030A0000E94443B80FF02C0599A01C05998809108
:1030B000C704882309F452C00E941516711009C074
:1030C0008FEE91E00E943E1680E00E947F300E94C9
:1030D00015164092B1038091C704813021F0809190
:1030E000C704823019F580E00E9422329091C70413
:1030F00081E0923009F080E00E94CB1C0E945E29A2
:103100000E94821381E0809338048093410480916F
:103110000304882321F00E946405A82E16C080E0D5
:103120000E94A6300E94360EA12C0FC0809103048D
:10313000882339F08091CA03811103C00E94EC0CEE
:1031400002C00E94360E44E1342E0E94510881E0F4
:103150000E9422321092C704772473948091210236
:10316000811129C080910304882329F18091B10342
:103170008F3F09F540912304509124046091250468
:10318000709126048091930390919403A0919503EC
:10319000B091960384179507A607B70760F480914E
:1031A000CA03882321F08091D503811104C0A110A6
:1031B00002C00E9401068091B1038F3F49F48091C3
:1031C0000304882329F08091CA03882309F4CEC020
:1031D00080914203662D0E94443B869DB02C1124B1
:1031E000DB1509F47AC080916102811103C08B2D37
:1031F0000E943A0E80910901873059F480911A0299
:10320000882339F00E947503882319F00E94EC048A
:1032100002C00E94540880910901883099F580917C
:10322000B1038250823070F5809143039091440342
:10323000C80ED91EE11CF11C1F5F103411F01111D2
:1032400011C0C701B60136E09695879577956795C9
:103250003A95D1F747E00E94AC3710E0C12CD12C51
:1032600076013BC0113021F480E40E940B1635C07A
:10327000183098F5E12FF0E0E95AFB4F80810E9469
:1032800018162BC00E94711A882339F18091CD0342
:10329000882319F18091430390914403C80ED91EED
:1032A000E11CF11C1F5F103111F0111116C0C70194
:1032B000B60124E096958795779567952A95D1F77D
:1032C0002091C8033091C90340E050E00E94643B64
:1032D00069017A01822E00E010E00E94711A8823B1
:1032E00099F0063088F431100FC00E9481158823B0
:1032F000F1F1053029F0602F882D0E94831702C05C
:103300000E94E20A0F5F33C00E94711A882379F18C
:103310008091BE03811104C08091B203882339F1EA
:103320000E9481158823A1F0332091F08FE083154E
:1033300058F0C1E0C30DE32DF0E0E15DFD4F808169
:103340000E9418163C2E13C00E94E20A312C0FC0B6
:103350000E948115882359F0311009C00E949D07F1
:10336000882329F00E943507382E01C0BD2E0E9407
:10337000BB2980910804811103C08091700080FFF7
:103380000E9463330E944532809152048F3F11F0B6
:103390000E94F6030E94D4118091550481110CC043
:1033A0000E943532C82F981641F08091580481113F
:1033B00004C00E94F63301C0C92D0E94B935809126
:1033C0003104882341F08091C704811104C0109218
:1033D00031040E94A630809180029091810297FD75
:1033E0000E94880B8091CA03882359F00E94993368
:1033F000882319F00E94590504C00E94B13381113D
:10340000F9CF80910304882359F08091CA03811178
:1034100007C08091800086FF03C080E00E94FC31DD
:103420000E94B11480E00E9421128091C804882378
:1034300049F180FF0FC08091B1038F3F59F4809113
:103440000304882339F0A11005C080912102811165
:103450000E9433298091C80481FF12C0109221027A
:103460008091230490912404A0912504B091260416
:103470008093930390939403A0939503B093960342
:103480001092C8048091D70381110E94322180914B
:103490007D02811107C080914A04811103C0DB2D98
:1034A0009C2EF7CD80917D02882319F00E941B0C81
:1034B00002C00E94E20A10924A048091B1038F3F39
:1034C00011F006E0ECCF3320E1F38091BE038111CF
:1034D00004C08091B2038823A1F30E943507382EDF
:1034E000F0CF8091B1038F3F39F094E0980F81E0E5
:1034F000923018F080E0089581E00895883080F4DB
:1035000090E0FC01EE0FFF1F8E0F9F1FFC01EA5899
:10351000FE4F80819181A281BC018A2F90E00895A5
:1035200061E070E080E090E00895CF93882389F017
:10353000C82F0E949E37843269F4EEE1F2E080E009
:103540009491C91721F08F5F31968B30C9F78C5D4C
:1035500001C080E0CF9108958A3010F4805D089515
:10356000843210F4895C0895E82FF0E0E650FE4FB5
:103570008491089584E090E00E94BF3DDC01CB017E
:10358000BF7781329D4CAB45B74071F080E790E04A
:103590000E94BF3D673672418B4E9C4D29F089E2F7
:1035A00092E00E943E16FFCF089590E00296880FA9
:1035B000991F880F991F0C94BF3D409104045091AE
:1035C0000504609106047091070488E590E00C946E
:1035D000DD3D4091D0035091D1036091D2037091B1
:1035E000D30384E590E00C94DD3D6091020483E018
:1035F00090E00E94CF3D4091D8035091D903609153
:10360000DA037091DB038CE790E00E94DD3D40918E
:10361000B3035091B4036091B5037091B60380E891
:1036200090E00E94DD3D6091080184E890E00E94F6
:10363000CF3D6091FC0385E890E00E94CF3D409132
:10364000BF035091C00360E070E088E490E00E9406
:10365000DD3D4091FE0350E060E070E08CE590E0DD
:103660000E94DD3D4091EC035091ED036091EE032B
:103670007091EF0380EC90E00C94DD3D83E090E0EE
:103680000E94B73D809302048CE790E00E94BF3D0A
:103690006093D8037093D9038093DA039093DB038C
:1036A00080E890E00E94BF3D6093B3037093B40341
:1036B0008093B5039093B60384E890E00E94B73DF1
:1036C0008093080188E490E00E94BF3D7093C0039E
:1036D0006093BF0385E890E00E94B73D8093FC03B0
:1036E0008CE590E00E94BF3D6093FE0380EC90E08B
:1036F0000E94BF3D6093EC037093ED038093EE0353
:103700009093EF030895CF92DF92EF92FF92CF93C1
:10371000DF93E0915904F0E0EE0FFF1FEC59FD4FED
:1037200025913491A8EEB3E00E948C3B6B017C01A3
:10373000C8E0D0E0B701A601CE010E94DD3D24968D
:10374000C834D105B9F7B701A6018CE790E00E9413
:10375000DD3DB701A60180E890E00E94DD3DB701A4
:10376000A60184E790E00E94DD3DB701A60184EA4E
:1037700090E00E94DD3DB701A60180EC90E00E9440
:10378000DD3D6091590486EC90E0DF91CF91FF9090
:10379000EF90DF90CF900C94CF3D8BEF8093B103EF
:1037A0000E94151689E492E00E943E161092590478
:1037B0000E943E0D1092C7040895CF93DF93EC0151
:1037C0000E941516CE010E943E16C0E0D0E060E0D7
:1037D000CE010E94CF3D2196C11584E0D807B9F7EC
:1037E00047E652E16BEE7CED80E790E00E94DD3D24
:1037F0004CEB52E060E070E080E590E00E94DD3D3F
:1038000040E65CE06CE971E084E590E00E94DD3D1B
:1038100040E05DE261E371E088E590E00E94DD3D1B
:103820004CE050E060E070E08CE590E00E94DD3D0F
:1038300044EF51E060E070E08CE690E00E94DD3DF6
:103840004CEB52E060E070E084EB90E00E94DD3DE4
:1038500043E650E060E070E088E790E00E94DD3DE4
:1038600045E250E060E070E088E690E00E94DD3DD7
:1038700040E050E860E070E088E490E00E94DD3DC8
:1038800066E084E890E00E94CF3D67E085E890E044
:103890000E94CF3D61E08CE990E00E94CF3D61E065
:1038A0008DE990E00E94CF3D61E08EE990E00E94BA
:1038B000CF3D4CEB52E060E070E088EA90E00E947F
:1038C000DD3D48E552E060E070E08CEA90E00E9467
:1038D000DD3D40E253E060E070E080EB90E00E946C
:1038E000DD3D40EE5EE260E070E088EB90E00E943B
:1038F000DD3D48EE53E060E070E08CEB90E00E942C
:10390000DD3D4CE251E060E070E080EA90E00E9432
:10391000DD3D4AE050E060E070E080E990E00E9428
:10392000DD3D47E050E060E070E084E990E00E9417
:10393000DD3D4CE350E060E070E088E990E00E94FB
:10394000DD3D44E650E060E070E08CE890E00E94ED
:10395000DD3D6FEF86EC90E00E94CF3D43E25DECF1
:103960006BE577E084E090E0DF91CF910C94DD3D52
:1039700084E090E00E94BF3DDC01CB01BF77833241
:103980009D4CAB45B74031F086E592E00E94DD1BCF
:103990000C9415160895CF93DF93C82F0E94B81C7E
:1039A000C1110E943E1B84E590E00E94BF3D6093E0
:1039B000D0037093D1038093D2039093D30388E50F
:1039C00090E00E94BF3D60930404709305048093CF
:1039D0000604909307048FE490E00E94B73D809323
:1039E000CC0380E590E00E94BF3D6093F4037093A8
:1039F000F5038093F6039093F70381E090E00E9433
:103A0000B73D8093E40382E090E00E94B73D80934D
:103A1000B90384EF93E00E94B73D8093E5038EE401
:103A200090E00E94B73D8093A8038CE690E00E944E
:103A3000BF3DEB0170930104609300048CE490E0BF
:103A40000E94B73D809303048DE490E00E94B73D4F
:103A50008093110480E690E00E94BF3D6093EB03E9
:103A600084E690E00E94BF3D6093C10388E690E049
:103A70000E94BF3D6093C70384E790E00E94BF3D72
:103A80006093F8037093F9038093FA039093FB0318
:103A900086E890E00E94B73D8093A90387E890E014
:103AA0000E94B73D8093CE038FE990E00E94B73D1E
:103AB0008093FD0388EB90E00E94BF3D7093F1037B
:103AC0006093F0038CEB90E00E94BF3D70930E0476
:103AD00060930D0480EA90E00E94BF3D7093E9037B
:103AE0006093E80380E990E00E94BF3D6093CF03BC
:103AF00084E990E00E94BF3D6093BB0388E990E0B9
:103B00000E94BF3D60930A048CE990E00E94B73D9B
:103B10008093BE038DE990E00E94B73D8093B2038D
:103B20008EE990E00E94B73D8093AA0384EC90E078
:103B30000E94B73D8093CB0385EC90E00E94B73D97
:103B40008093CD038CE890E00E94BF3D7093C90341
:103B50006093C80387EC90E00E94B73D8093F30325
:103B6000E29730F482E390E09093010480930004A4
:103B70008091000490910104873B934030F086EBE4
:103B800093E0909301048093000489E08093810086
:103B900084EB90E00E94BF3D6E3581E0780710F421
:103BA0006EE571E09B0140E050E06091040470918B
:103BB000050480910604909107040E94643B3093B1
:103BC00089002093880080918800909189009695C3
:103BD000879590938B0080938A0088E790E00E94FD
:103BE000BF3D83E6861B8823A9F020918A0030918F
:103BF0008B0040918A0050918B0094E05695479538
:103C00009A95E1F7241B350B30938B0020938A00A3
:103C10008150E9CF8091FD03811110922804DF913A
:103C2000CF910895E0910901EB3028F4F0E0E559D7
:103C3000FE4F8081089580E00895E091B1038E2FBA
:103C400090E08A30910520F5FC01EA5BFF4F0C946F
:103C5000863B8EEC95E01AC085EC95E017C081ECB0
:103C600095E014C08BEB95E011C083EB95E00EC09E
:103C70008CEA95E00BC086EA95E008C08CE995E0F7
:103C800005C08DE895E002C08EE795E00C943E16E5
:103C9000089580910901853029F481E09091B10364
:103CA000983009F080E00895CF92DF92EF92FF9272
:103CB0000F931F938091B7039091B8030E94BF3D6B
:103CC00020910901223059F52091B103243039F5B2
:103CD000611520E872078105910588F400E010E87D
:103CE00020E030E068017901C61AD70AE80AF90A2B
:103CF000C701B60147E00E94AC378DE207C070589B
:103D00008109910947E00E94AC378BE28093590406
:103D10001F910F91FF90EF90DF90CF900895409109
:103D2000D4031F910F91FF90EF90DF90CF900C94F0
:103D3000AC37EF92FF920F931F93CF93DF938C01D9
:103D4000EB017A010E94491E882311F180911E0423
:103D50002AE0622F0E94443B805D80935904905D6D
:103D600090935A048AE380935B04809129040E9413
:103D7000443B805D80935C04905D90935D04109261
:103D80005E0486E08093D40382E08093AB032DC071
:103D90008091B10390E0F701E80FF91F249120937F
:103DA000AB03FE01E80FF91FC491C093D403880F41
:103DB000991FD801A80FB91F8D919C919093B803BA
:103DC0008093B703223019F40E94541E0EC0213094
:103DD00041F44C2F50E0BC0189E594E00E94A73DDE
:103DE00004C00E94B73D80935904DF91CF911F9189
:103DF0000F91FF90EF900C94C10D86E795E00E9423
:103E00003E168091B10360E08F5F0E949D1682E0B4
:103E10008093AB038BE08093D4038091B10390E057
:103E20000296880F991F880F991F9093B80380936B
:103E3000B7030E94BF3D4BE00E94AC370C94C10D0C
:103E4000843010F082E3089584E60895843010F001
:103E500042E301C044E64093D403843038F424E6BE
:103E6000829FC001112488539F4F0BC090E004979C
:103E700052E3589F9001599F300D1124C901885A6F
:103E80009D4F9093B8038093B70350E06091B703C0
:103E90007091B80389E594E00C94A73D8091B1033B
:103EA0008C3099F484E695E00E943E1682E080937F
:103EB000AB0383E08093D40388E890E09093B80349
:103EC0008093B7030E94541E27C08D30A1F48CE567
:103ED00095E00E943E161092AB0381E08093D403DC
:103EE00086E890E09093B8038093B7030E94B73DB3
:103EF0008093590411C08DE695E00E943E16809192
:103F0000B10360E08F5F0E949D1681E08093AB0358
:103F10008091B1030E94261F0C94C10DE091B10362
:103F20008E2F90E088309105F0F4FC01E05BFF4FAC
:103F30000C94863B83E595E014C08DE495E011C0B8
:103F400087E495E00EC08DE395E00BC089E395E032
:103F500008C080E395E005C088E295E002C08EE1EC
:103F600095E00E943E1644EC52E06CEC72E08CED61
:103F700091E00C94991EE091B1038E2F90E08A306D
:103F8000910520F5FC01E85AFF4F0C94863B83E134
:103F900095E01AC087E095E017C08CEF94E014C05C
:103FA00080EE94E011C08FEE94E00EC084EE94E0B9
:103FB0000BC087ED94E008C08AEC94E005C08DEB5F
:103FC00094E002C081EB94E00E943E1640EB52E088
:103FD0006AEB72E088EC91E00C94991E8091B10339
:103FE000823099F038F4882369F08130C1F48AE98D
:103FF00094E013C0843079F058F0853081F48FE676
:1040000094E00BC085EA94E008C08FE894E005C016
:1040100085E894E002C08BE794E00E943E1644EAF3
:1040200052E06AEA72E08CEB91E00C94991E90E009
:104030008930910508F5FC01EE59FF4F0C94863B41
:1040400088E694E017C083E694E014C089E594E024
:1040500011C083E594E00EC08DE494E00BC083E4CE
:1040600094E008C088E394E005C08BE294E002C0CD
:1040700082E294E00C943E1608958091B1030E9470
:10408000172044E952E06CE972E08CEA91E00C946C
:10409000991EE091B1038E2F90E08930910508F5CB
:1040A000FC01E559FF4F0C94863B87E194E017C073
:1040B0008CE094E014C081E094E011C086EF93E0BE
:1040C0000EC089EE93E00BC08CED93E008C08FEC3E
:1040D00093E005C085EB93E002C082EC93E00E9480
:1040E0003E168091B103883099F480E40E940B164B
:1040F00086EA93E00E943E1682E08093AB0383E061
:104100008093D40343E060E070E0CB010C94AC37C3
:1041100042E852E06BE872E08AE991E00C94991E63
:10412000E091B1038E2F90E08D30910568F5FC0190
:10413000EC58FF4F0C94863B8CE993E023C080E958
:1041400093E020C083E893E01DC086E793E01AC0A7
:104150008EE693E017C083E693E014C08AE593E00F
:1041600011C082E593E00EC089E493E00BC080E4C7
:1041700093E008C084E393E005C088E293E002C0C6
:104180008FE193E00E943E1680911A02882349F045
:104190008091B103863018F40E94DE0302C00E94B1
:1041A0007D038091B103863040F446E752E06CE72E
:1041B00072E08EE891E00C94991E80911A028111B0
:1041C00007C080E40E940B1681E193E00C943E1638
:1041D0000895CF92DF92EF92FF92CF93C1E0C09308
:1041E0000804C0900404D0900504E0900604F09008
:1041F0000704C701B60120E03AE040E050E00E9429
:10420000643B3093BD032093BC03C701B6012AE091
:1042100030E040E050E00E94643B20931004209383
:10422000B3001092DC03109285001092840010926B
:10423000D703EAE7F0E08081877F8083C0936F0037
:1042400010928100C093B1001092B2008FEF9FEFE7
:1042500090930C0480930B04CF91FF90EF90DF902C
:10426000CF90089580E40E940B162091C3033091F3
:10427000C4034091C5035091C603AAE0B0E00E9478
:10428000A23B4AE00E94AC37E9E5F4E08EE281838C
:1042900086818583878186831782CF010E943216AB
:1042A00084E492E00E943E160C94E92010926F0084
:1042B000EAE7F0E080818860808310920804089526
:1042C0008FEF0E9469368091B1038230B1F028F4FB
:1042D000882349F0813051F008958430A9F080F0AE
:1042E0008530C1F0089589E093E002C080E093E05A
:1042F0000E943E1610922804089585EF92E002C0B5
:104300008AEE92E00C943E1680EE92E00E943E16F9
:104310000C94E92084ED92E00E943E1682E08093A6
:10432000AB0380EC90E09093B8038093B7038CE0EC
:104330008093D4030E94541E0C94C10D0E94151644
:10434000809109018A3031F08F5F0E9424168EE23D
:104350000E941816909109018091B1039A3011F4CE
:10436000893039F060E08F5F0E949D1680E20E94E4
:104370001816E09109018E2F90E08B309105C8F45A
:10438000FC01EF57FF4F0C94863B0C941D1E0C94C0
:10439000FD1E0C944E1F0C948E1F0C94BB1F0C948E
:1043A000EE1F0C943D200C9449200C9490200C940A
:1043B00060210895E0917E02F0917F02E75AFB4F61
:1043C00080818B3211F48DE201C08BE280830895ED
:1043D0008091AB038330E1F080910901823029F4B0
:1043E0009091B103963069F413C08330B9F4909181
:1043F000B103992359F1993069F081E09530A9F41E
:1044000025C0992319F1933039F0953071F404C027
:1044100081E0089582E0089588E00895853039F4B8
:1044200081E09091B103913089F080E0089581306E
:1044300031F48091B1038D30C1F783E60895863061
:10444000A1F781E09091B103943079F708958091BC
:104450000901883059F48091B103833019F48FEF4A
:104460000C946936843011F40C945621089589E532
:1044700094E00E9476386093EC037093ED03809390
:10448000EE039093EF0382E00C94A630CF92DF927C
:10449000EF92FF920F931F93CF93DF93E82E082F95
:1044A00010E0E801C75ADB4F8881893341F50E944B
:1044B000491E811122C0E11002C0F12C24C0FF244A
:1044C000FA94FE0CCF2CD12CFF2051F0F601E75AC4
:1044D000FB4F80810E946738811102C0FA94F2CFAD
:1044E000F601E75AFB4F80810E946738882329F341
:1044F0008F2D0E944622882301F380E301C08F5F45
:104500008883FF24F39480917E0290917F020817A4
:10451000190779F00E94081690E0005C1F4F801781
:10452000910721F080E48E0D0E940B1688810E9475
:1045300018168F2DDF91CF911F910F91FF90EF9063
:10454000DF90CF900895CF92DF92EF92FF920F937A
:104550001F93CF93DF93E82E082F10E0E801C75A8E
:10456000DB4F8881803341F50E94491E811122C0B2
:10457000E11002C0F12C24C0FF24FA94FE0CCF2CD1
:10458000D12CFF2051F0F601E75AFB4F80810E94A9
:104590006738811102C0FA94F2CFF601E75AFB4F57
:1045A00080810E946738882329F38F2D0E94A322DF
:1045B000882301F389E301C081508883FF24F394A9
:1045C00080917E0290917F020817190779F00E946E
:1045D000081690E0005C1F4F8017910721F080E4DF
:1045E0008E0D0E940B1688810E9418168F2DDF9168
:1045F000CF911F910F91FF90EF90DF90CF90089592
:1046000080915904811102C084E007C09091B103E8
:10461000843040F4933021F487E080935904089566
:1046200088E0FBCF933011F4883071F30895CF9375
:10463000DF9380910904882309F4A3C080E00E94DD
:10464000C80A8091AB03813009F477C028F082302A
:10465000E1F0833009F090C080915904811103C0CA
:104660000E94E82101C08150809359048091090182
:10467000823041F48091B103853011F0833011F420
:104680000E9400230E94C10D77C0809109018230F1
:1046900069F48091B103843049F480917E02909155
:1046A0007F02892B19F40E94DA2104C080917E02D6
:1046B0000E94A3220E94491E8823C9F080915904B8
:1046C000893319F482E38093590480915904823329
:1046D00039F480915A04843318F083E380935A04A8
:1046E00080915C04893319F485E380935C040E9413
:1046F000081640917E0250917F02282F30E0CA01B7
:10470000805C9F4F2817390721F080E4840F0E94B6
:104710000B16E0917E02F0917F02E75AFB4F8081F9
:104720000E94181680910901883031F58091B103FB
:10473000853011F50E9437221FC0E0917E02F09172
:104740007F02E75AFB4F80810E94951A811101C0B8
:104750008FE2C0917E02D0917F0281500E94AC1AFC
:10476000C75ADB4F8883E0917E02F0917F02E75ABF
:10477000FB4F80810E94181681E0DF91CF910C944D
:10478000C80A0E94121E9091B103981798F40E94D3
:1047900027228091B103811104C00E94121E8093D0
:1047A000B1038091B10381508093B103DF91CF9128
:1047B0000C949E21DF91CF910895CF93DF93809148
:1047C0000904882309F4A4C080E00E94C80A8091EB
:1047D000AB03813009F478C028F08230E9F08330EF
:1047E00009F091C0C0915904CF5FC09359040E9451
:1047F000E8218C1710F4109259048091090182303D
:1048000041F48091B103853011F0833011F40E949E
:1048100000230E94C10D77C080910901823069F4A4
:104820008091B103843049F480917E0290917F029F
:10483000892B19F40E94DA2104C080917E020E9423
:1048400046220E94491E8823C9F08091590483336F
:1048500019F480E38093590480915904823339F428
:1048600080915A04843318F080E380935A04809135
:104870005C04863319F480E380935C040E9408167C
:1048800040917E0250917F02282F30E0CA01805C67
:104890009F4F2817390721F080E4840F0E940B16E0
:1048A000E0917E02F0917F02E75AFB4F80810E94E7
:1048B000181680910901883031F58091B103853057
:1048C00011F50E9437221FC0E0917E02F0917F0215
:1048D000E75AFB4F80810E94951A8F5F8F3208F054
:1048E00080E0C0917E02D0917F020E94AC1AC75A2C
:1048F000DB4F8883E0917E02F0917F02E75AFB4F05
:1049000080810E94181681E0DF91CF910C94C80A33
:1049100080E00E94C80A0E942722C091B103CF5FA5
:10492000C093B1030E94121EC81710F01092B10379
:10493000DF91CF910C949E21CF93DF938091AB03B5
:10494000813009F07AC080917E0290917F02FC0153
:10495000E75AFB4F20812F3759F521E0280F30917E
:10496000D403231748F4A22FB0E0A75ABB4F4C91B1
:1049700011974C932F5FF5CF009799F0208121116B
:1049800010C0019790937F0280937E0280917B02FA
:1049900090917C02009729F0019790937C0280937C
:1049A0007B02E0917E02F0917F02E75AFB4F1DC02F
:1049B0002E37F9F42091F2032083A091D4034FEF16
:1049C0004A0F242F30E08217930748F4275A3B4FB1
:1049D000E90121975881E90158834150F2CF80E2E3
:1049E0008083B0E0A85ABB4F1C9280818093F20371
:1049F00022C02630A1F410927F0210927E02109203
:104A00007C0210927B02109259041092F20380E40F
:104A10000E940B160E9408160E944D160CC02730EB
:104A200061F48091F20380838091D40390E09093AD
:104A30007F0280937E0281E001C080E0DF91CF9110
:104A40000895CF92DF92EF92FF920F931F93809180
:104A5000AB03813081F4E0917E02F0917F02E75A4E
:104A6000FB4F808192E8980F923018F08650823088
:104A700010F40E949C2410927F0210927E021092E9
:104A80007C0210927B02109209040E941B1780E0A6
:104A90000E94C80A0E94C10D0E94491E8823E1F0AD
:104AA00060915C04660F6056862F880F880F680F30
:104AB00080915D048053680F80915904880F80565F
:104AC000982F990F990F890F90915A04905340E0B5
:104AD000890F0E94B32961C02091AB03223009F0F5
:104AE00049C0809109018230F9F48091B10384308A
:104AF000D9F48AE594E00E947638209159042D3249
:104B000069F400E010E820E030E068017901C61A9D
:104B1000D70AE80AF90AB701A6010CC0AB01BC012B
:104B200050586F4F7F4F06C089E594E00E94763859
:104B3000AB01BC01209109012630A9F42091B103F9
:104B4000283089F44131510561057105D1F58AE3B9
:104B500092E00E94DD1B1F910F91FF90EF90DF907C
:104B6000CF900C94CD1B8091B7039091B8030E9415
:104B7000DD3D13C08091B7039091B803213049F413
:104B80004091D40350E0BC0189E594E00E94C53D0A
:104B900004C0609159040E94CF3D84E090E00E94DF
:104BA000BF3D97FD0EC043E25DEC6BE577E884E026
:104BB00090E01F910F91FF90EF90DF90CF900C94B9
:104BC000DD3D1F910F91FF90EF90DF90CF90089502
:104BD0000E949C24811149C02091AB0380917E02E8
:104BE00090917F02213041F4FC01E75AFB4F208174
:104BF000211102C020E220830097E1F4E0917E02BF
:104C0000F0917F02E75AFB4F80818093F2032DC021
:104C100080917E0290917F020097A9F0FC01E75AF3
:104C2000FB4F80810E94673881110DC080917E0208
:104C300090917F02019790937F0280937E028091F2
:104C4000AB03823029F320917E0230917F02809164
:104C50007B0290917C022817390710F40197FBCF53
:104C600090937C0280937B02C9CF0E94C10D81E0AA
:104C70000C94C80ACF93C82F0E949C24811144C071
:104C80002091AB0380917E0290917F022130C1F48C
:104C9000FC01E75AFB4F2081211112C020E2208342
:104CA0000FC0E0917E02F0917F02E75AFB4F8081B6
:104CB0000E94673881110DC080917E0290917F0221
:104CC000019690937F0280937E028091AB038230A5
:104CD00041F380917E0290917F0220917B0230917E
:104CE0007C02AC01421B530B4031510518F02F5F81
:104CF0003F4FF7CF30937C0220937B02FC01E75AB1
:104D0000FB4F80818093F2038091D40390E0AC014B
:104D10004150510920917E0230917F0224173507BE
:104D200050F0CC2319F0CF910C9421250297909349
:104D30007F0280937E028091AB039FEF980F9230A9
:104D400080F4E0917E02F0917F02E75AFB4F908160
:104D5000911107C0823011F480E301C080E28083AA
:104D60000AC08091EA03882339F0E0917E02F09135
:104D70007F02E75AFB4F11820E94C10D81E0CF9163
:104D80000C94C80A80E40E940B1683E50E94181652
:104D900080E20E9418168091BA03893048F480E2BC
:104DA0000E9418168091BA038F5F0E94241605C0D6
:104DB0008091BA038F5F0E94271680E20E94181626
:104DC0008091BA030E94D51A0E94440B80E20E948F
:104DD00018168CE40C9418161F93CF93DF9380E47D
:104DE0000E940B1680910F0460E08F5F0E949D1659
:104DF0008EE20E94181680E20E94181680910F041D
:104E00000E94261FC9E5D4E01991111107C00E9424
:104E10000816DF91CF911F910C944D160E94081631
:104E20008035A8F7812F0E941816EECF2091FC0341
:104E3000283078F430E0F901EE0FFF1F2E0F3F1FEE
:104E4000F901EA58FE4F208131814281642FA90186
:104E500004C041E050E060E070E02091BF03309179
:104E6000C003882339F0420F531F403187EA5807A7
:104E700068F408C0C901841B950BAC01413F98E55B
:104E8000590720F05093C0034093BF030E94250BA5
:104E900081E08093310408959091FE03882321F0EE
:104EA000933638F49F5F03C0923018F0915090937E
:104EB000FE030E94340B0C948213909159048823B2
:104EC00031F09F5F993050F01092590409C0911150
:104ED00004C088E08093590403C091509093590412
:104EE0000C943E0D882361F08091BA038F5F80930C
:104EF000BA038091BA03803171F41092BA030BC0E7
:104F00008091BA03882321F08091BA03815001C0B7
:104F10008FE08093BA030C94C226882361F08091BD
:104F20000F048F5F80930F0480910F048C3071F415
:104F300010920F040BC080910F04882321F0809100
:104F40000F04815001C08BE080930F040C94EC2679
:104F500080910204813059F48091BA034091B303E7
:104F60005091B4036091B5037091B6030AC080916B
:104F7000BA034091D8035091D9036091DA0370913C
:104F8000DB0390E00296880F991F880F991F0C94FD
:104F9000DD3D80910204813069F48091BA030E9462
:104FA000D51A6093B3037093B4038093B5039093C1
:104FB000B6030CC08091BA030E94D51A6093D8033F
:104FC0007093D9038093DA039093DB0381E080939D
:104FD000380480E00C94A6300E94272280910904B6
:104FE000882319F00E94212514C0809109018A307C
:104FF00051F08093B1038AE0809309010E949E21C1
:105000000E94DE0306C081E08093C7048EE1809396
:10501000550480E00E94961280E00C942832809122
:105020000904882319F081E00C943A268091090143
:105030008A3071F48091B103893021F40E94F51A0D
:105040000C94EC27809309011092B1030C949E21DB
:10505000873051F48091B103863068F080911A0254
:1050600081114CC00C947D03883029F48091B103E8
:10507000853009F043C08091AB03813039F49091C1
:105080005904911103C08093EA0304C01092EA030B
:10509000813011F40E946A168091AB03823051F482
:1050A0008091D403833031F481E090E090937F02CB
:1050B00080937E0281E08093090480E48093C203A0
:1050C00080910901883059F48091B103853099F4B9
:1050D00080E00E94223282E00E94A6300CC086301E
:1050E00051F48091B103883031F40E94C10D0E94C7
:1050F00008160E944D1681E00C94C80A08951F926C
:105100000F920FB60F9211248F938091DC038F5F63
:105110008093DC038F910F900FBE0F901F90189516
:105120001F920F920FB60F9211242F933F934F931C
:105130005F936F937F938F939F93AF93BF93EF93FF
:10514000FF93809108048823F9F080910B049091DB
:105150000C04019690930C0480930B04892B19F492
:1051600087E08093810020910B0430910C048091A2
:10517000BC039091BD032817390741F4809170005A
:1051800082608093700002C00E946333FF91EF91B0
:10519000BF91AF919F918F917F916F915F914F914F
:1051A0003F912F910F900FBE0F901F9018951F9257
:1051B0000F920FB60F9211242F933F938F939F93CB
:1051C000AF93BF9380910804882341F180910B0431
:1051D00090910C04019690930C0480930B04892BFE
:1051E00011F010928100209184003091850080910F
:1051F000DC0390E0A0E0B0E0DC0199278827820F73
:10520000931FA11DB11D8093C3039093C403A0936A
:10521000C503B093C60381E08093D70380917000EB
:105220008D7F80937000BF91AF919F918F913F913F
:105230002F910F900FBE0F901F9018959091C10362
:10524000209129043091EB03892F281710F0830F48
:10525000FCCF809318048C3310F09093180481E0F5
:1052600080932102089580E40E940B1680911E0411
:105270000E9427168AE30E941816809129040E9432
:1052800027168AE30E94181680911D040E94271693
:1052900080E20E94181680E20E9418168CE30E9499
:1052A000181680E20E941816809118040E94271692
:1052B00080E20E94181680E20C941816CF92DF92BA
:1052C000EF92FF92CF93DF9316BC109223041092BB
:1052D0002404109225041092260460910404709115
:1052E000050480910604909107046B017C012AE07B
:1052F000F694E794D794C7942A95D1F7C0921904ED
:10530000D0921A04E0921B04F0921C04EB01D370BB
:10531000D0932B04C0932A04C0921F04D09220047F
:10532000E0922104F092220420E038EC40E050E0CA
:105330000E94643BC20ED31EE41EF51EC0921204EE
:10534000D0921304E0921404F0921504D093170441
:10535000C093160487E2DF91CF91FF90EF90DF902A
:10536000CF900C949D156093290480931E04409364
:105370001D040C945E298F929F92AF92BF92CF92A0
:10538000DF92EF92FF92CF93DF9396B580910B025D
:1053900081112AC097FF3FC081E080930B0280916A
:1053A0002804882369F080910901883049F48091AC
:1053B000B103823028F4809128048150809328041E
:1053C00080915504882319F0815080935504809171
:1053D00027048F5F80932704809154048823D9F099
:1053E00081508093540417C097FD15C010920B0292
:1053F0004091230450912404609125047091260467
:105400005F5F6F4F7F4F409323045093240460935A
:10541000250470932604C0902304D0902404E090C7
:105420002504F0902604CC24C90ED11CE11CF11CEB
:10543000C0922304D0922404E0922504F092260422
:105440008091120490911304A0911404B09115045A
:105450000097A105B10509F4B8C08C159D05AE05EE
:10546000BF0508F0B2C01092530410922704609157
:10547000190470911A0480911B0490911C04C0912E
:105480001604D091170420912A0430912B04C20FE6
:10549000D31F80901F0490902004A0902104B0900E
:1054A0002204860E971EA81EB91E9E01232F3327A5
:1054B00026952695820E931EA11CB11C80921F0476
:1054C00090922004A0922104B092220422E330E0C2
:1054D00040E050E00E94643BDA01C901880D991D4B
:1054E000AA1DBB1D8093120490931304A09314046F
:1054F000B0931504D370D0931704C093160481E0C1
:1055000088169104A1048FEFB806B0F08091930340
:1055100090919403A0919503B09196038C199D09E5
:10552000AE09BF098093930390939403A0939503CE
:10553000B09396030E945E298091D503882319F0C9
:1055400081508093D50380912804882329F080918D
:10555000280481508093280480911D048F5F8C3330
:1055600019F080931D0416C010921D048091290427
:105570008F5F8C3319F0809329040CC0109229049A
:1055800080911E048F5F883119F080931E0402C041
:1055900010921E048091C804982F91609093C804C3
:1055A000209129049091180429130FC09091210291
:1055B000992359F090911104992321F090911D04A1
:1055C000992319F083608093C804DF91CF91FF90F5
:1055D000EF90DF90CF90BF90AF909F908F90089505
:1055E000CF93DF93D82FC62F80EC0E9429038D2FF5
:1055F0000E943B03811109C08C2F0E943B03811143
:1056000006C00E94330380E003C083E001C084E051
:10561000DF91CF9108954F925F926F927F928F9218
:105620009F92AF92BF92CF92DF92EF92FF920F9331
:105630001F93CF93C82F462E6701780149015A0165
:1056400087E0880C991CAA1CBB1C8A95D1F7C50160
:10565000B401A70196010E94643BCA01B901512C13
:10566000612C712C27E0440C551C661C771C2A9574
:10567000D1F722E0521A61087108460E571E681EC3
:10568000791EA70196010E94343B861A970AA80A40
:10569000B90A6D2D8C2F0E94F02A6C2D81E08C0FA1
:1056A0000E94F02AD301C20188279927A370BB2743
:1056B000BD018827992782E08C0F0E94F02A652D72
:1056C00083E08C0F0E94F02A642D84E08C0F0E94EE
:1056D000F02ACC24DD248FE0E822FF244CE0F6946D
:1056E000E794D794C7944A95D1F7D501C401882788
:1056F0009927AF70BB276C2D6A2B85E08C0F0E9419
:10570000F02A692D86E08C0F0E94F02A682D87E030
:105710008C0FCF911F910F91FF90EF90DF90CF9062
:10572000BF90AF909F908F907F906F905F904F90C1
:105730000C94F02ACF92DF92EF92FF920F93CF93C7
:10574000DF93C82FD22F4450510961097E4F6A015F
:105750007B0187E0CC0CDD1CEE1CFF1C8A95D1F789
:1057600060E08C2F0E94F02A61E081E08C0F0E94A3
:10577000F02AD701C60188279927A370BB276D2F70
:10578000602B6A2B82E08C0F0E94F02A6D2D83E043
:105790008C0F0E94F02A6C2D84E08C0F0E94F02A5E
:1057A00060E085E08C0F0E94F02A60E086E08C0FBC
:1057B0000E94F02A60E087E08C0FDF91CF910F917B
:1057C000FF90EF90DF90CF900C94F02ACF93C82FEA
:1057D0000E94140360E88C2F0E94F02ACF910C9451
:1057E0001903CF93C82F0E941403CC2371F060E2F9
:1057F0008CE30E94F02A60E48BEB0E94F02A63E4C1
:1058000082E10E94F02A60E008C060E08BEB0E9419
:10581000F02A82E10E94E62B64E083E00E94F02AF5
:10582000CF910C941903EF92FF920F931F93CF9394
:10583000C82F0E941403809137048C17A8F540915B
:1058400030042C2F30E090E04423C9F08901081B7C
:10585000190BC801092E000CAA0BBB0B40913D048B
:1058600050913E0460913F04709140048A019B0175
:10587000081B190B2A0B3B0BD901C80130C0A90129
:10588000481B590BCA01092E000CAA0BBB0B4091F7
:105890003304509134046091350470913604840FC0
:1058A000951FA61FB71F34C0C817D8F54091300404
:1058B0002C2F30E090E0821B930B092E000CAA0BDA
:1058C000BB0B4423A9F040913D0450913E046091EC
:1058D0003F0470914004840F951FA61FB71F80934B
:1058E0003D0490933E04A0933F04B093400428C02D
:1058F0004091330450913404609135047091360422
:105900008A019B01081B190B2A0B3B0BD901C8010B
:105910008093330490933404A0933504B0933604F9
:105920000FC08C130DC06FE682E10E94F02AC09375
:105930003704CF911F910F91FF90EF900C941903B2
:10594000E0903D04F0903E0400913F04109140042B
:105950002091330430913404409135045091360441
:105960006091320482E20E940B2BDDCFCF92DF9256
:10597000EF92FF929B01AC0160912C0470912D0479
:1059800080912E0490912F040E94343B6093420436
:10599000709343048093440490934504C090D003D3
:1059A000D090D103E090D203F090D303A7019601E9
:1059B0000E94643B20933204462F572FBC018FEF87
:1059C0009FEFAFE0B0E080933D0490933E04A0933E
:1059D0003F04B093400424E180E090E0DC01440FF8
:1059E000551F661F771F880F991FAA1FBB1F4C15D5
:1059F0005D056E057F0528F04C195D096E097F096C
:105A00008160215061F78093330490933404A09314
:105A10003504B0933604FF90EF90DF90CF90089557
:105A20004F925F926F927F928F929F92AF92BF92AE
:105A3000CF92DF92EF92FF920F931F93CF93DF935A
:105A4000CDB7DEB728970FB6F894DEBF0FBECDBF37
:105A500029013A01F50120912C0430912D04409147
:105A60002E0450912F04D6010E94A23B4B015C01F1
:105A7000CF01A0E0B0E089839A83AB83BC83C801E7
:105A8000B701A50194010E94643B2D833E834F839F
:105A900058879B01AC0169817A818B819C810E942E
:105AA000343BA50194010E94643B49015A012D81B8
:105AB0003E814F81588569817A818B819C810E94CA
:105AC000343B95018401060F171F281F391F0093CF
:105AD0003D0410933E0420933F043093400485E13D
:105AE00040E050E0BA01769567955795479540FE9E
:105AF00004C0400F511F621F731F76946794579420
:105B00004794815081F74093330450933404609359
:105B1000350470933604411551056041710538F420
:105B200081E0011511052041310508F080E028963B
:105B30000FB6F894DEBF0FBECDBFDF91CF911F919E
:105B40000F91FF90EF90DF90CF90BF90AF909F901C
:105B50008F907F906F905F904F9008954F925F92DB
:105B60006F927F92AF92BF92CF92DF92EF92FF92AD
:105B70000F931F93CF93DF93CDB7DEB72D970FB65B
:105B8000F894DEBF0FBECDBF2B013C010E94140371
:105B900060E079EE84EA95E3A30192010E94643B00
:105BA00029833A834B835C83DA01C9018170992789
:105BB000AA27BB2789879A87AB87BC8720FD03C0AC
:105BC000DA01C90107C089819A81AB81BC81019743
:105BD000A109B10980932C0490932D04A0932E0465
:105BE000B0932F041D8660912C0470912D04809138
:105BF0002E0490912F04A30192010E94343B611561
:105C00007644834C934208F46EC08D8581118EC01A
:105C1000C301B2010E94B62C8091330490913404E8
:105C2000A0913504B09136048D839E83AF83B887ED
:105C3000E090D003F090D1030091D2031091D303F0
:105C4000A12CBB24B39457E7C52EDD24D3949C012B
:105C5000AD01C301B2010E94102D882329F01092DA
:105C6000300491E09D87BFCF60914204709143045E
:105C700080914404909145042091D0033091D10348
:105C80004091D2035091D3030E94643BA12CBB24CA
:105C9000B39437E7C32EDD24D3947B018C012D818F
:105CA0003E814F815885C301B2010E94102D882387
:105CB00031F0A1E0A0933004B1E0BD8794CF809192
:105CC0002C0490912D04A0912E04B0912F040297E2
:105CD000A109B10980932C0490932D04A0932E0464
:105CE000B0932F0480CF9D85911120C089859A851E
:105CF000AB85BC85892B8A2B8B2B29F489819A81D2
:105D0000AB81BC8107C089819A81AB81BC8101973D
:105D1000A109B10980932C0490932D04A0932E0423
:105D2000B0932F04C301B2010E94B62CE0903D0451
:105D3000F0903E0400913F04109140042091330400
:105D4000309134044091350450913604609132040E
:105D500082E20E940B2B40912C0450912D04609103
:105D60002E0470912F0400E020E08AE30E949A2B19
:105D700060EA81EB0E94F02A109237042D960FB64C
:105D8000F894DEBF0FBECDBFDF91CF911F910F9171
:105D9000FF90EF90DF90CF90BF90AF907F906F908B
:105DA0005F904F900C9419033F924F925F926F92C5
:105DB0007F928F929F92AF92BF92CF92DF92EF929B
:105DC000FF920F931F93CF93DF93C82F6A017B013C
:105DD000452B462B472B41F40E94E62B81E0C13135
:105DE00009F47BC180E079C14090D0035090D10389
:105DF0006090D2037090D3030E94140380E8C81609
:105E000081EDD80680EFE80688E0F80608F07CC04F
:105E1000809109018830A9F485E08093B10360E0A6
:105E200079EE84EA95E3A70196010E94643B49015B
:105E30005A01253833404105510508F03FC0312C47
:105E40005BC0C11482E1D8068AE7E806F10408F4D1
:105E50001EC1C1148BE1D80687EBE806F10408F4F3
:105E60001CC180ECC81681EED80684EEE806F10469
:105E700008F419C180ECC8168AEED80681E2E8065B
:105E800081E0F80608F415C180E8C81681EBD80651
:105E90008FE4E80681E0F80608F411C180E8C8162E
:105EA0008AEBD8068CE8E80681E0F80608F40DC114
:105EB0008CE1882E912CA12CB12C0CC107E0CC0CCC
:105EC000DD1CEE1CFF1C0A95D1F760E079EE84EA38
:105ED00095E3A70196010E94643B49015A012538C8
:105EE00033404105510530F014E8812E13E0912E26
:105EF000A12CB12CD0E73D2E80FE0DC081E0881A88
:105F00009108A108B10807C0B4E08B2E912CA12CF8
:105F1000B12CDCE0E0C0D0E0A7019601C501B401DE
:105F20000E94343BA30192010E94643BE22FF4E102
:105F300020E030E0A901660F771F881F991F220F0C
:105F4000331F441F551F641575058605970528F0F6
:105F500064197509860997092160F15061F7CC240D
:105F6000C39481EF8E0F8C3458F0C12C60E88C2FD5
:105F70000E94F02AC03109F086C060E881E181C04A
:105F8000C03139F0AAE36A2EB0E2DB2E12E2712EA4
:105F900005C07AE2672ED12CFAE17F2EE090390419
:105FA000F0903A0400913B0410913C048091E4038A
:105FB0008E149F04A006B10621F490910C0298174C
:105FC00069F091E0909338048092390490923A04F9
:105FD000A0923B04B0923C0480930C02EE24EA941D
:105FE000FE2C0FE010E06E2F872D0E940B2B0D2F43
:105FF000232DB501A401862D0E949A2BC031F1F406
:10600000232DB501A40182E30E949A2B60E085EA6A
:106010000E94F02A682D86EA0E94F02ACD2DCF64D6
:106020006C2F80E10E94F02A8091E403813019F402
:106030006D2D6F6501C06C2F81E105C0C23129F45F
:106040006D2D6F6482E10E94F02A82E2781207C00F
:10605000809138048823B9F060E881EB12C08AE1AE
:10606000781211C080910801843020F080913804AA
:10607000882349F060E281EB0E94F02A10923804F4
:1060800002C00E94F02A0E9419038C2D26C05EE7F0
:10609000852E912CA12CB12C1DC044E5842E912C71
:1060A000A12CB12C17C030E4832E912CA12CB12C43
:1060B00011C020E3822E912CA12CB12C0BC098E2B0
:1060C000892E912CA12CB12C05C082E2882E912C16
:1060D000A12CB12CD0E0312C1FCFDF91CF911F919B
:1060E0000F91FF90EF90DF90CF90BF90AF909F9077
:1060F0008F907F906F905F904F903F900895CF93D7
:10610000C82F0E941403CC2351F060E48BEB0E9453
:10611000F02A62E083E00E94F02A63E409C060E0B4
:106120008BEB0E94F02A64E083E00E94F02A6FE487
:1061300080E10E94F02ACF910C9419030E9414036D
:1061400060E083E00E94F02A0C941903CF92DF9262
:10615000EF92FF92CF93823071F44091EC03509113
:10616000ED036091EE037091EF0380E10E94D42E65
:1061700080934104B1C0C091E403813009F044C070
:1061800084EA90E00E94BF3D6B017C018091B103E5
:10619000863059F44091F4035091F5036091F60371
:1061A0007091F703C130A1F41CC0883019F48CEA57
:1061B00090E007C0893019F480EB90E002C088EAD3
:1061C00090E00E94BF3DAB0160E070E0C13049F457
:1061D000D701C601841B950BA60BB70BAC01BD0103
:1061E00004C04C0D5D1D6E1D7F1D80E10E94D42EEC
:1061F00080934104B701A60182E1CF91FF90EF9017
:10620000DF90CF900C94D42E80910304882359F012
:106210004091F8035091F9036091FA037091FB03E8
:106220006A017B0131C040910204411109C0C09054
:10623000D803D090D903E090DA03F090DB030EC0CE
:106240003091B3032091B4039091B5038091B603CC
:10625000C32ED22EE92EF82E413071F4B701A601DB
:106260005058610971098091BF039091C003480F94
:10627000591F611D711D08C04091D8035091D90369
:106280006091DA037091DB038091F4039091F50340
:10629000A091F603B091F703C13029F4480F591FBC
:1062A0006A1F7B1F04C0481B590B6A0B7B0B80E1E4
:1062B0000E94D42E80934104B701A60182E10E947E
:1062C000D42E80914104811107C0CF91FF90EF90AF
:1062D000DF90CF900C94360ECF91FF90EF90DF902F
:1062E000CF9008951D9912C080916B008F7D80938F
:1062F0006B008091B200865A8093B40010924804DB
:10630000BA9A8091700084608093700008951F9203
:106310000F920FB60F9211242F933F934F935F93D9
:106320006F937F938F939F93AF93BF93EF93FF935D
:106330008091B2008F5B8093B400809148048830D4
:1063400090F4809148048F5F8093480480914904C1
:106350008695809349041D9B1AC0809149048068EA
:106360008093490414C0809170008B7F80937000EB
:10637000E0914604F0914704309719F08091490468
:106380000995D89A80916B00806280936B00FF9191
:10639000EF91BF91AF919F918F917F916F915F919D
:1063A0004F913F912F910F900FBE0F901F90189516
:1063B00010927000EBE6F0E080818F7D808308957D
:1063C00021E42093B4009093470480934604E0E7CF
:1063D000F0E080818B7F808383E08093B1002D9AF1
:1063E000E8E6F0E0808181608083D89AEBE6F0E017
:1063F0008081806280830895882391F080910304D6
:10640000882321F08091CA03882351F0219A80E4E7
:106410008093800080916F00846080936F00089566
:10642000219880916F008B7F80936F008091800016
:106430008F7B809380000895882311F02B9A089514
:106440002B980895882311F0289A08952898089584
:10645000882311F02A9A08952A98089589B186FB15
:10646000882780F991E0892708958091570480FF5B
:1064700002C084E001C080E09091570491FD8E5FDE
:106480009091570492FD8F5F0895CF92DF92EF9223
:10649000FF92CF93DF939091B1039F3F39F48091A6
:1064A0000304882319F080E880930A0180910A018F
:1064B000803809F401C138F080910A01815080933D
:1064C0000A0181E006C080910A018F5F80930A0172
:1064D00080E09F3F09F06FC09091A3039111ECC041
:1064E0009091570490FF10C090910801811105C050
:1064F000933008F458C0915004C0973008F053C04E
:106500009F5F909308014FC090910204913019F061
:10651000C8EDD3E002C0C3EBD3E0811123C0C88033
:10652000D980EA80FB80809108010E947E1A6C1558
:106530007D058E059F0588F4809108010E947E1AD2
:10654000C880D980EA80FB80A7019601261B370B03
:10655000480B590BDA01C9011FC0188219821A822F
:106560001B821EC0809108010E947E1AC880D980BB
:10657000EA80FB80DC01CB018C0D9D1DAE1DBF1D93
:10658000811531EE930735EFA30735E0B30720F00F
:106590008FEF90EEA5EFB5E088839983AA83BB8344
:1065A00081E080933104DF91CF91FF90EF90DF90F5
:1065B000CF900C94360E9E3F41F4DF91CF91FF9027
:1065C000EF90DF90CF900C9472279A3F41F4DF91C7
:1065D000CF91FF90EF90DF90CF900C948D279D3F4F
:1065E00029F59091A303911167C09091570490FFF2
:1065F00015C09091FC03811104C0943038F0915083
:1066000003C0983018F49F5F9093FC03DF91CF9103
:10661000FF90EF90DF90CF900C94E20ADF91CF9142
:10662000FF90EF90DF90CF900C9416279C3F41F4A1
:10663000DF91CF91FF90EF90DF90CF900C944C279B
:106640009B3F41F4DF91CF91FF90EF90DF90CF908F
:106650000C945D27909109049923E1F090915704DF
:1066600090FF18C09091AB039150923098F488231A
:1066700049F080E0DF91CF91FF90EF90DF90CF90D5
:106680000C943A26DF91CF91FF90EF90DF90CF905E
:106690000C94E825882341F0DF91CF91FF90EF9093
:1066A000DF90CF900C94DD23DF91CF91FF90EF909E
:1066B000DF90CF900C941723DF91CF91FF90EF9054
:1066C000DF90CF9008950E942E3229B1922F90959D
:1066D000991F9927991F30911402831304C0309198
:1066E0001302391729F130911202332329F0309126
:1066F000130239131092120230911202311114C098
:10670000882391F03091140231110EC031E03093A2
:10671000120227FD04C020910A012F5F03C02091BF
:106720000A01215020930A018093140290931302CE
:1067300008958091B903811105C09091E5039230CD
:1067400078F409C08091A803882329F083B185FBE0
:10675000882780F903C083B18295817091E08927F1
:10676000089583B1807290911102891739F1809355
:106770001102809153048F3F21F08F5F8093530467
:106780001DC08091CE03811119C08091CA0381116F
:1067900015C080910304811111C080911A028111EA
:1067A0000DC00E94711A811104C08091B10387FD50
:1067B00005C081E08093CE030E94360E8091B9031C
:1067C000811105C09091E5039D7F79F408C0809107
:1067D000A803882321F083B18295817004C083B11E
:1067E00085FB882780F991E0892708950F931F93EF
:1067F000CF93DF93D82F8091CA03811103C081E02A
:106800000E9421120E943532C82F882329F08093DC
:10681000100281E0809358048091B1038C3F19F4F9
:10682000D11164C144C08D3F99F4D1115FC1C1FD44
:1068300041C0C0FF5BC180E090E89093C0038093AB
:10684000BF0383E08093C70481E0809331044EC18D
:106850008B3F71F4CC2309F484C10E94831B82E036
:106860008093C7041092B1038AE0809309013EC16E
:106870008E3F79F4D1113AC1C1FF03C00E94A8270D
:1068800019C0C0FF03C00E94C92714C0C2FF2EC197
:1068900011C08A3F99F4D11129C1C1FF02C080E023
:1068A00003C0C2FF04C081E00E94E7051FC1CC23E2
:1068B00009F457C183E08093C70418C187FD10C055
:1068C000D11114C180910F02811110C1C1FF03C009
:1068D0000E940F280BC1C0FF09C10E94EC2706C10E
:1068E0008091CA03811104C080910304882349F078
:1068F000C0FFFCC0809155048111F8C00E94590569
:10690000F5C0CC2399F1D0910E02D11128C0A091ED
:10691000E803B091E9032091190430911A044091E1
:106920001B0450911C040E94A23B28EE33E040E07F
:1069300050E00E94643B8091230490912404A09134
:106940002504B0912604820F931FA41FB51F8093C6
:106950004B0490934C04A0934D04B0934E0480914B
:106960000F02811103C0DF5FD0930E0280910E02EF
:106970008230E1F040914B0450914C0460914D0401
:1069800070914E0400912304109124042091250459
:1069900030912604401751076207730748F4CC234F
:1069A00011F083E003C0882319F081E080930D0289
:1069B00080910D02882309F499C09091100291FFF3
:1069C00019C0833039F40E94121E8093B1030E94D3
:1069D000DD237BC0823031F48DEF8093B1030E94C0
:1069E000250B73C0813031F48CEF8093B1030E948A
:1069F000340B6BC020915404392F31702223C9F01D
:106A0000332309F44AC08130A1F44091B30350917B
:106A1000B4036091B5037091B6034093D8035093CB
:106A2000D9036093DA037093DB0393E09093C70478
:106A30002FC0332391F1813089F4809102048F5F5C
:106A4000833018F48093020402C01092020483E0A1
:106A50008093C70481E08093310437C0222309F476
:106A60004DC0823009F052C08091D8039091D90373
:106A7000A091DA03B091DB038093B3039093B40346
:106A8000A093B503B093B60383E08093C70481E07D
:106A9000809331041092540418C092FF16C08130C4
:106AA00061F4809108018F5F883008F084E0809362
:106AB000080181E080934A0408C08250823028F4A3
:106AC0008AEF8093B1030E94EC2610920E0210927E
:106AD0000D028FEF9FEFDC0180934B0490934C04E9
:106AE000A0934D04B0934E0410921002C0930F0275
:106AF000CC23C9F180E00E94BB3835C0823031F42C
:106B00008EEF8093B1030E94C226DFCF833029F637
:106B10004091D8035091D9036091DA037091DB035F
:106B20000091B3031091B4032091B5033091B603E3
:106B30000093D8031093D9032093DA033093DB0337
:106B40004093B3035093B4036093B5037093B603BB
:106B50008093C70481E0809331048CE480935404D3
:106B6000B4CF10920F028C2FDF91CF911F910F9114
:106B7000089580914B0490914C04A0914D04B091E4
:106B80004E04409123045091240460912504709197
:106B9000260484179507A607B70770F480E00E94C3
:106BA000F6338FEF9FEFDC0180934B0490934C04FE
:106BB000A0934D04B0934E04089586E08093B100F5
:106BC00081E08093700008955E9A5F9A2C9A2D9AC6
:106BD000209A229AE8E6F0E0808182608083ECE6E9
:106BE000F0E08081886080838FEF9FEFDC018093ED
:106BF0004B0490934C04A0934D04B0934E0480E05A
:106C00000E94FC310C94DD35E0E7F0E080818E7F5E
:106C1000808308951F920F920FB60F9211248F93C5
:106C2000199B05C0809182008068809382008F91BB
:106C30000F900FBE0F901F9018951F920F920FB6D6
:106C40000F9211242F933F934F935F936F937F93F2
:106C50008F939F93AF93BF93EF93FF930E94C53899
:106C600080915604811107C081E00E94F6338111A2
:106C700002C010925804FF91EF91BF91AF919F9184
:106C80008F917F916F915F914F913F912F910F90D5
:106C90000FBE0F901F9018951F920F920FB60F9274
:106CA00011248F938FEE80937A0080917A0083FD78
:106CB00005C080917A00886080937A0080915704A3
:106CC0008061809357048F910F900FBE0F901F909B
:106CD00018958F3FA9F480910901883021F48091A3
:106CE000B103833051F080911A02882341F081E092
:106CF0009091B103963019F403C081E001C080E0A7
:106D000020917C002F7030E0482F50E02417350789
:106D100049F090917C00907F890F80937C0081E006
:106D200080934F0408951F920F920FB60F92112473
:106D30002F933F934F935F936F937F938F939F9383
:106D4000AF93BF93EF93FF9380914F04882319F083
:106D500010924F047CC080917C008F70823069F467
:106D6000809178009091790090689093810280934F
:106D700080028FE0809328042CC080917C008F706B
:106D8000833049F580915704887F80935704809120
:106D9000780090917900833D934020F080915704D2
:106DA000816015C08091780090917900833593407F
:106DB00020F08091570484600AC0809178009091FF
:106DC0007900853F914028F080915704826080933C
:106DD00057048FEF3AC0E091420380917800909180
:106DE0007900F0E0EE0FFF1FEE57FD4F9183808397
:106DF000809142038F5F80934203809142038036EB
:106E000011F4109242038091570484FF09C083E07B
:106E10000E946936809157048F7E8093570417C073
:106E200080912804811113C080911A0281110FC032
:106E30008091FD03811108C080910901883039F4E7
:106E40008091B103823018F482E00E946936FF918C
:106E5000EF91BF91AF919F918F917F916F915F91D2
:106E60004F913F912F910F900FBE0F901F9018954B
:106E700020E0611571058105910539F060FD2F5FF6
:106E80009695879577956795F4CF822F81700895B1
:106E9000262F269526952695820F911DFC0180812F
:106EA00090E070E0609570956770772702C09595C7
:106EB00087956A95E2F781700895262F2695269585
:106EC0002695FC01E20FF11D70E0609570956770EA
:106ED000772721E030E001C0220F6A95EAF7808130
:106EE000282B20830895262F26952695820F911D05
:106EF000FC01808190E070E0609570956370772769
:106F0000660F771F02C0959587956A95E2F78370A3
:106F10000895262F26952695FC01E20FF11D80810C
:106F200070E06095709563707727660F771F01C0DA
:106F3000440F6A95EAF7482B4083089590ED980F27
:106F40009A3030F09FEB980F9A3120F487530895D0
:106F5000892F089584E20895CF93C42F20910901C9
:106F60002230B9F42091B103243099F461152AEC50
:106F700072072AE982072BE3920710F02DE201C085
:106F80002BE220935A0420E03AEC4AE95BE30E94AA
:106F9000643B20E0611531EE730735EF830735E080
:106FA000930728F0715E854F95402F5FF3CF205DEA
:106FB00020935B0420E0603836E9730738E98307E3
:106FC000910530F060587649884991092F5FF3CFD9
:106FD000205D20935C0420E0603432E473073FE0DE
:106FE0008307910530F0605472448F4091092F5F00
:106FF000F3CF205D20935D042CE220935E0420E01B
:10700000603A36E8730731E08307910530F0605A43
:107010007648814091092F5FF3CF205D20935F0474
:1070200020E0603137E273078105910530F060514F
:107030007742810991092F5FF4CF205D209360048E
:1070400020E0683E33E073078105910530F0685E0B
:107050007340810991092F5FF4CF205D2093610473
:107060002CE22093620420E06436710581059105CD
:1070700030F064567109810991092F5FF5CF205DC9
:107080002093630420E06A3071058105910530F09A
:107090006A507109810991092F5FF5CF205D209316
:1070A0006404605D6093650410926604EEE0F0E0B5
:1070B000EC1BF109E75AFB4FA9E5B4E080E08C171F
:1070C00021F091919D938F5FFACFCF91089590ED2C
:1070D000980F81E09A3008F080E0089590ED980FC5
:1070E0009A3010F087530895892F08958F929F92B8
:1070F000AF92BF92CF92DF92EF92FF92CF93DF9346
:10710000EC01E0E0DE01AE0FB11D8C91882311F09F
:10711000EF5FF8CFE150C12CD12C7601812C912C5E
:1071200054018394EF3FD1F0DE01AE0FB11DAC915D
:1071300080ED8A0F8A3080F4B0E0D097A5019401E9
:107140000E94AD3BC60ED71EE81EF91EAAE0B0E0B5
:107150000E94A23B4B015C01E150E4CFC701B601A4
:10716000DF91CF91FF90EF90DF90CF90BF90AF90E5
:107170009F908F900895F894A895E0E6F0E088E15C
:1071800080838BE4808378940895F894A89584B7DD
:10719000877F84BFE0E6F0E0808188618083108291
:1071A00078940895FC0180818154823170F481814A
:1071B0008154823150F4828180538A3030F483814B
:1071C00080538A3010F480E0089586E008952F926D
:1071D0003F924F925F926F927F928F929F92AF9267
:1071E000BF92CF92DF92EF92FF920F931F93CF93B4
:1071F000DF93CDB7DEB7E0970FB6F894DEBF0FBED2
:10720000CDBF47E050E068EE73E089E594E00E946E
:10721000A73D809159049FEB980F9A3110F410E02C
:1072200009C00E9467388111FACF809159048032D9
:10723000B1F315E080915A049FEB980F9A3128F032
:107240000E946738811101C015E080915B040E94A3
:107250006738811101C015E080915C049FEB980FA5
:107260009A3118F0803209F015E080915D049FEBAF
:10727000980F9A3118F0803209F015E080915E0481
:107280009FEB980F9A3118F0803209F0AAC01111C3
:1072900094C1809159040E949E37282F30E0A4E2C7
:1072A000B0E00E948C3B6B017C0180915A040E94EB
:1072B0009E37A7019601280F311D411D511DAAE0DF
:1072C000B0E00E94A23B6B017C0180915B040E94B4
:1072D0009E37A7019601280F311D411D511D2BA777
:1072E0003CA74DA75EA70CE514E06FE5E62E64E031
:1072F000F62EF80181918F010E949E37E82FABE1B5
:10730000B0E02BA53CA54DA55EA50E94A23BDC01EB
:10731000CB010A97A109B1099C01AD012E0F311DC6
:10732000411D511D2BA73CA74DA75EA7E016F106F6
:1073300001F745E050E06FEE73E089E594E00E94CC
:10734000A73D89E594E00E94D238182F811135C1FC
:10735000809159040E949E37082F80915B040E94FF
:107360009E37202F30E02A50310946EF4203D001EA
:10737000439FB00D1124AD54BF4FA81BB10924EB9E
:1073800030E00E949B3B4B015C0180915A040E94BB
:107390009E37082F80915C040E949E37202F30E09A
:1073A0002A5031096AE0629F6001639FD00C11246A
:1073B0000D2C000CEE08FF08C80ED11CE11CF11CBE
:1073C0008C0C9D1CAE1CBF1C2091C7032D3358F4A0
:1073D000822F0E94443B992341F09B7F933019F404
:1073E00004C015E0EAC017E0E8C08091EB039FEF0E
:1073F000980F9E3180F480FD0EC08091F80390912B
:10740000F903A091FA03B091FB03892B8A2B8B2BF4
:1074100021F412E0D2C013E0D0C087E0880C991CA0
:10742000AA1CBB1C8A95D1F7822F90E0A0E0B0E0A7
:10743000805C9F4FAF4FBF4F6C017D01C80CD91CC2
:10744000EA1CFB1CFE017696CE018B965F01119221
:107450008E179F07E1F7FE013196EFA7F8AB119267
:10746000AE16BF06E1F74BE1842E912C00E0412CD3
:10747000512C32015FE1252E312C0C3168F48BA5A3
:107480009CA5ADA5BEA5082C04C0B695A79597955B
:1074900087950A94D2F713C0023398F48EEE800FCA
:1074A000A101481B5109CA01A701960104C05695C4
:1074B0004795379527958A95D2F7DA01C9018170EA
:1074C00001C080E0440C551C661C771C480E511C02
:1074D000611C711CC301B20161757375807D927F5F
:1074E0000E943837882329F0602F660FC5010E945B
:1074F0005D37C301B20167747C738176947E0E940C
:107500003837882331F0602F660F6F5FC5010E9406
:107510005D370F5F31E0831A9108013509F0ADCF77
:10752000912C812C97E0E92EF12CCC24C394D12C02
:1075300080E090E000E0282D30E0A901082E02C094
:10754000559547950A94E2F740FF0AC0A701481BEA
:10755000590BB60102C0660F771F4A95E2F7062B5A
:1075600001968830910549F7023A60F4692DC5010A
:107570000E944837882329F0602F8FA598A90E9480
:107580005D379394839471EA791590F600E0602F4B
:107590008FA598A90E944837F82E602F8BE091E0C4
:1075A0000E944837FF0C4F2D480F602F89EC94E064
:1075B0000E9489370F5F023A51F7812FE0960FB68C
:1075C000F894DEBF0FBECDBFDF91CF911F910F9119
:1075D000FF90EF90DF90CF90BF90AF909F908F90F3
:1075E0007F906F905F904F903F902F900895CF9332
:1075F00080912402823A90F581110CC06091F803C9
:107600007091F9038091FA039091FB030E94AE2DD3
:107610001092A3036091240289EC94E00E947337D6
:10762000C82F0E94132C81E00E9496128BE00E94CA
:107630000B1660E0809124020E949D1680E20E9459
:1076400018168C2F0E94241680E20E941816809132
:1076500024028F5F8093240280E004C080E00E94B7
:10766000961281E0CF910895DB018F939F930E9442
:10767000A23BBF91AF91A29F800D911DA39F900D42
:10768000B29F900D11240895991B79E004C0991FB1
:10769000961708F0961B881F7A95C9F7809508956C
:1076A000AA1BBB1B51E107C0AA1FBB1FA617B70728
:1076B00010F0A61BB70B881F991F5A95A9F7809544
:1076C0009095BC01CD010895A1E21A2EAA1BBB1B07
:1076D000FD010DC0AA1FBB1FEE1FFF1FA217B3079E
:1076E000E407F50720F0A21BB30BE40BF50B661FB4
:1076F000771F881F991F1A9469F760957095809578
:1077000090959B01AC01BD01CF010895EE0FFF1FC5
:107710000590F491E02D0994A29FB001B39FC001A0
:10772000A39F700D811D1124911DB29F700D811DAD
:107730001124911D08950E948C3BB7FF0895821B70
:10774000930B08950E948C3BA59F900DB49F900DC4
:10775000A49F800D911D11240895B7FF0C94A23BA6
:107760000E94A23B821B930B08955058BB27AA2767
:107770000E94CD3B0C94A53C0E94973C38F00E949F
:107780009E3C20F039F49F3F19F426F40C94943C6D
:107790000EF4E095E7FB0C948E3CE92F0E94B63C7A
:1077A00058F3BA17620773078407950720F079F436
:1077B000A6F50C94D83C0EF4E0950B2EBA2FA02D14
:1077C0000B01B90190010C01CA01A0011124FF278E
:1077D000591B99F0593F50F4503E68F11A16F04089
:1077E000A22F232F342F4427585FF3CF4695379588
:1077F0002795A795F0405395C9F77EF41F16BA0B4D
:10780000620B730B840BBAF09150A1F0FF0FBB1FFA
:10781000661F771F881FC2F70EC0BA0F621F731F43
:10782000841F48F4879577956795B795F7959E3FA0
:1078300008F0B0CF9395880F08F09927EE0F979531
:10784000879508950E94BE3C88F09F5798F0B92F05
:107850009927B751B0F0E1F0660F771F881F991F85
:107860001AF0BA95C9F714C0B13091F00E94D83C13
:10787000B1E008950C94D83C672F782F8827B85F23
:1078800039F0B93FCCF3869577956795B395D9F7DD
:107890003EF490958095709561957F4F8F4F9F4FE7
:1078A0000895E89409C097FB3EF4909580957095F3
:1078B00061957F4F8F4F9F4F9923A9F0F92F96E93C
:1078C000BB279395F695879577956795B795F111B1
:1078D000F8CFFAF4BB0F11F460FF1BC06F5F7F4F4E
:1078E0008F4F9F4F16C0882311F096E911C0772360
:1078F00021F09EE8872F762F05C0662371F096E869
:10790000862F70E060E02AF09A95660F771F881F37
:10791000DAF7880F9695879597F9089597F99F67F5
:1079200080E870E060E008959FEF80EC0895002407
:107930000A941616170618060906089500240A94D4
:1079400012161306140605060895092E0394000C5A
:1079500011F4882352F0BB0F40F4BF2B11F460FFE9
:1079600004C06F5F7F4F8F4F9F4F089557FD905812
:10797000440F551F59F05F3F71F04795880F97FBF3
:10798000991F61F09F3F79F08795089512161306AD
:107990001406551FF2CF4695F1DF08C016161706DC
:1079A0001806991FF1CF8695710561050894089511
:1079B000E894BB2766277727CB0197F908950E94A3
:1079C000F23C0C94A53C0E94973C38F00E949E3CEF
:1079D00020F0952311F00C948E3C0C94943C1124CF
:1079E0000C94D93C0E94B63C70F3959FC1F3950F5F
:1079F00050E0551F629FF001729FBB27F00DB11D33
:107A0000639FAA27F00DB11DAA1F649F6627B00DC2
:107A1000A11D661F829F2227B00DA11D621F739FAB
:107A2000B00DA11D621F839FA00D611D221F749FB9
:107A30003327A00D611D231F849F600D211D822F00
:107A4000762F6A2F11249F5750409AF0F1F0882327
:107A50004AF0EE0FFF1FBB1F661F771F881F915054
:107A60005040A9F79E3F510580F00C948E3C0C9439
:107A7000D93C5F3FE4F3983ED4F3869577956795BC
:107A8000B795F795E7959F5FC1F7FE2B880F911D7E
:107A90009695879597F9089519F416F40C94943CEB
:107AA0000C94923D0E94BE3CB8F39923C9F3B6F3FF
:107AB0009F57550B87FF0E94A03D0024A0E640EA97
:107AC000900180585695979528F4805C660F771F33
:107AD000881F20F026173707480730F4621B730B06
:107AE000840B202931294A2BA69517940794202529
:107AF00031254A2758F7660F771F881F20F0261771
:107B00003707480730F4620B730B840B200D311DCF
:107B1000411DA09581F7B901842F9158880F969542
:107B2000879508959F3F31F0915020F48795779580
:107B30006795B795880F911D9695879597F9089544
:107B400091505040660F771F881FD2F70895DC01CF
:107B5000CB01FC01F999FECF06C0F2BDE1BDF89A58
:107B6000319600B40D9241505040B8F70895F999FC
:107B7000FECF92BD81BDF89A992780B50895A6E100
:107B8000B0E044E050E00C94A93DDC01CB0103C01F
:107B90002D910E94D03D41505040D0F70895262F9E
:107BA000F999FECF1FBA92BD81BD20BD0FB6F894E2
:107BB000FA9AF99A0FBE01960895242F0E94D03D9B
:107BC000252F0E94D03D0C94E53D0E94CF3D272FEC
:087BD0000C94D03DF894FFCFA6
:107BD8000A000A005F83EC3F060A80C08E25E02574
:107BE80002CD1A1AA92C6A2093B34705301AC60089
:107BF800DFCFC7C3C1C0D0D8DCDEF9E8EAF4FCE2C5
:107C0800F6E0F8E7F5E4FBFAF7E6EDF2F0FDF1E16E
:107C1800F3E9EBECEFD2D18C95B332440033440056
:107C28004E6F002D2D002D20732D00524D4300471F
:107C38005341004747410047535600100E080A06B3
:107C480009090D06000A80969840420FA086011087
:107C58002700E80300F401006400000A0000A40003
:107C6800A800AC00B00054005800A0009F00B80065
:107C7800BC00C400C5008C00F50300004C004D009A
:107C8800740060006400E803EF036800900094004B
:107C980098009C009D009E0002005C004E006C0055
:107CA800C7004F008700B4007800F40303007C008D
:0C7CB8008000840048008500010050009E
:00000001FF
